:10000000004000203D4A00007D4A00007F4A000079
:1000100000000000000000000000000000000000E0
:10002000000000000000000000000000814A000005
:100030000000000000000000834A0000854A000024
:10004000874A0000874A0000B94E0000874A000036
:10005000874A000000000000874A0000874A00002D
:10006000874A00007D510000874A0000874A00004F
:10007000874A0000874A0000874A0000874A00003C
:10008000874A0000ED520000874A0000874A0000BE
:10009000874A0000874A0000874A0000874A00001C
:1000A000874A0000874A00000000000000000000AE
:1000B0000000000000000000000000000000000040
:1000C00010B5064C2378002B07D1054B002B02D02E
:1000D000044800E000BF0123237010BD1404002079
:1000E0000000000098A80000044B10B5002B03D0BE
:1000F0000349044800E000BF10BDC04600000000F6
:100100001804002098A80000164B002B00D1144BB7
:100110009D46402292029A1A924600218B460F4633
:100120001348144A121A08F03AF90F4B002B00D06A
:1001300098470E4B002B00D0984700200021040068
:100140000D000D48002802D00C4800E000BF08F068
:10015000E5F82000290004F0C7FE08F0B9F8C04611
:100160000000080000400020000000000000000027
:100170001404002068270020000000000000000098
:1001800002000120104004D1042A01D9106800099E
:1001900070470020FCE710B50400FFF7F1FF0028CE
:1001A00009D001388000031D22181279002A02D0DC
:1001B00001309842F8D110BD0122096810B51142F2
:1001C00001D0002903DA102000F082F910BD491097
:1001D000062002F017F8F9E7096810B5CB0701D53A
:1001E000002903DA102000F073F910BD4910033123
:1001F00089100022052002F005F8F6E770B50D68B9
:10020000AB0729D1042D27D90F232A684E68134044
:10021000062B0BD12800FFF7B3FF0123984201DA28
:1002200000200AE09A00AE500133F7E7052B13D106
:10023000F30703D4132000F04BF970BD7610FF2EA6
:10024000F8D82800FFF79CFF2C1D80002018A04242
:10025000E6D926700134FAE70B2000F039F9DFE720
:1002600070B50C681120E30712D54D68AB072BD190
:10027000042D29D90F262B6864101E40062E0DD19F
:10028000002C04DD2800FFF77BFFA04203DA1220D8
:1002900000F01EF901E0A400605970BD331F012B6E
:1002A00012D82800FFF76CFF8000042E02D128002E
:1002B000FFF771FF002CEADDA042E8DB01202C19DA
:1002C000E3785B001843E8E70B20E1E7F8B501238A
:1002D0000D6811201D4214D003244E6834402CD1E7
:1002E000042E2AD90F2332686D108F681340062B15
:1002F0000ED1002D04DD3000FFF742FFA84203DAE3
:10030000122000F0E5F802E0AD00AF512000F8BD8A
:10031000052B12D1002DF3DD3000FFF731FF8000F7
:10032000A842EDDB01231F4201D11320E9E77F1032
:10033000FF2FFAD87519EF70E8E70B20E1E708689E
:1003400010B5830717D1042815D90F23026813406D
:10035000062B03D1FFF714FF430004E0052B05D162
:10036000FFF70EFFC3000120184310BD042B02D17C
:10037000FFF711FFF0E70B2000F0AAF8F5E7000007
:1003800002000120104001D0501070470D22014B97
:100390001A70FAE75404002002000120104004D132
:1003A000042A01D91068000970470020FCE770B5E5
:1003B0000D000400FFF7F0FF06002800FFF7ECFF38
:1003C0000023864207D1231DB6009E1904351A006A
:1003D0009E4202D80123180070BD2978127801339B
:1003E00001358A42F3D00023F5E70000F0B585B06F
:1003F0000393019002912D4E2D4B002A02D0022230
:100400003270013A00251A601B68F554019B9D4229
:1004100001DB05B0F0BD029AAB00D058244B1C683C
:10042000C8239B0037191C1B0123184206D0214A00
:1004300043102100380008F05BFB09E01E4A002849
:1004400002D004281BD11D4A2100380008F050FBBF
:10045000300008F0B1FB164A039B1060002B0CD053
:10046000019B013BAB4208DD154B984205D8431C6C
:100470001360202232540022F2540135C6E70428CA
:1004800010D90F2302681340042B04D101F0F6FEAB
:100490000C4A0300CDE7062B05D1FFF77DFF0A4A82
:1004A0000300C6E70123094AC3E7C04655040020FC
:1004B00078070020459B0000189B00001E9B000051
:1004C0001F030000E9A10000239B0000349B0000F3
:1004D000014B1870002070475404002070B501F0E3
:1004E000EFFC094C0100251D1F22280008F06BFBC2
:1004F000280008F061FB0423043080080001184341
:100500002060200070BDC04630040020C368F0B5F4
:100510009D00836889B05D19030018330693036951
:10052000069A9F00069B0390DF19436901939B0085
:10053000D3180293CD4B1B78002B26D17F222B683A
:10054000CB491C1213409B005B58043501929F4617
:10055000039B587803F072FB0023039A137027E083
:10056000C24B1B78002B10D12B68019A1C12134030
:10057000BF4A9B009B580435E9E7069B3A1DD11AF8
:10058000BA4BD82928DD1A221A70039BB74C9B68F6
:1005900021780193EA1A039B92109B7812021A4366
:1005A000039B587803F052FB0023039A23701370C7
:1005B000039B069A9B680193ED1A039BAD10DD60C7
:1005C000069BFE1A039BB6101E61029B9B1A039AA0
:1005D0009B10536109B0F0BD1B783C60002B01D02B
:1005E0001700D2E72B6801991C120B40A0499B0011
:1005F0005B5817000435AAE7069B3A1DD11A9B4B9E
:10060000D82902DD1A221A70BFE728681B78291D35
:100610003860002B02D017000D00B6E76B68019917
:100620001C120B4092499B005B58170008358EE75F
:10063000069B3A1DD11A8D4BD82902DD1A221A7059
:10064000A3E7A4001B782C193C60002B01D01700F5
:100650009BE72B6801991C120B4085499B005B5856
:100660001700043573E7069B3A1DD11A7F4BD82932
:1006700002DD1A221A7088E77E49A40061581B78AF
:100680003960002B01D017007FE72B6801991C12FD
:100690000B4077499B005B581700043557E7043F30
:1006A000744B3A68A400E250704B1B78002B00D0CA
:1006B0006BE72B68019A1C1213406D4A9B009B58F4
:1006C000043544E76B4BA400E058FFF759FE043FA4
:1006D00006003868FFF754FE36180120654B760097
:1006E0000643E650614B1B78002B00D04DE72B688A
:1006F000019A1C1213405E4A9B009B58043526E762
:10070000069B3A1DD11A594BD82902DD1A221A70BC
:100710003BE70698029C0121A04202D221000C393D
:1007200009681B783960002B01D017002DE72B6872
:1007300001991C120B404E499B005B581700043571
:1007400005E7069B3A1DD11A484BD82902DD1A222B
:100750001A701AE70699029881420FD203000C3BE7
:100760001B6845495B106418E41AA40023583B60D9
:100770003E4B1B78002B05D0170006E71821197097
:100780000023F4E72B6801991C120B4038499B00A9
:100790005B5817000435DAE6069B029A934219D299
:1007A00013000C3B1B68344A043FA4185B10E31A87
:1007B000029A39689B0099502C4B1B78002B00D073
:1007C000E3E62B68019A1C121340294A9B009B58B0
:1007D0000435BCE61822254B1A70EDE7069B029AF9
:1007E00093422DD2244B3E1FE31814000C3C04937B
:1007F0002368049A5B10D31A029A9B009858FFF75B
:10080000BFFD07903068FFF7BBFD2468049B6410B0
:100810001C1B079BA4001F1801207F00029B07439D
:10082000E7503700114B1B78002B00D0ADE62B684A
:10083000019A1C1213400E4A9B009B58043586E611
:1008400018220A4B1A70EDE7069B3A1DD11A074B86
:10085000D82902DD1A221A7097E60299A40061587D
:100860001B783960002B09D017008EE65404002055
:1008700018990000AC240020FDFFFF3F2B68019970
:100880001C120B40D8499B005B58170004355EE6EC
:10089000043F029B3A68A400E250D44B1B78002B23
:1008A00000D072E62B68019A1C121340CE4A9B00BE
:1008B0009B5804354BE6029BA4001C192368043F97
:1008C00038685E10FFF75CFD36180120C74B7600D4
:1008D0001B7806432660002B00D056E62B68019A51
:1008E0001C121340C04A9B009B5804352FE6069B00
:1008F000A4003F1BBD4CBB420CD82378002B00D07A
:1009000043E62B68019A1C121340B74A9B009B5880
:1009100004351CE6B64801F025FC2378002B00D0F6
:1009200033E62B68019A1C121340AF4A9B009B5878
:1009300004350CE6A300ED18002C00DA38E6AB4BCA
:100940001B78002B00D020E62B68019A1C12134064
:10095000A54A9B009B580435F9E5043F3B68042BEE
:1009600004D1A300ED18002C00DA21E69F4B1B7880
:10097000002B00D009E62B68019A1C1213409A4AFA
:100980009B009B580435E2E5043F3B68042B06D0EE
:10099000A200AD18002C02DA002B00D108E6934B20
:1009A0001B78002B00D0F0E52B68019A1C12134035
:1009B0008D4A9B009B580435C9E53A1F13685B10AC
:1009C000013B002B06DD01215B00A4000B432D1928
:1009D0001360EDE5854B17001B78002B00D0D4E5A4
:1009E0002B68019A1C1213407F4A9B009B580435C8
:1009F000ADE53A00069B0C32D31AD82B03DD1A2240
:100A00007A4B1A70C1E5FF2361005B001940FE3B81
:100A1000FF3B1943396003990698896824120491B1
:100A20006D1A0399AD1089782D020D4302999D40EE
:100A3000091A891099401D430B43BB60039B7D60DD
:100A40009C70E4B26B4BE4000292E358039A93600B
:100A5000664A1278002A03D008331D00029F94E5ED
:100A60001D00019A9B680C351C1213405E4A9B00C6
:100A70009B58029F6BE53B1F1C68029A069B9342A2
:100A80002FD10A20E3070ED4A30715D1042C13D9C4
:100A90000F2322681340042B11D1200001F0EEFB3C
:100AA00008F08AF80630643002F0B2FD00280FD159
:100AB000043D069B02937BE50720042CF3D0200025
:100AC000431E9841FA234042FF3318400730EAE7BB
:100AD000039B2100587803F0CBF80023039A13708E
:100AE000E7E7029B029A0C3B1B6803995B109B0093
:100AF000D31A0C3B1C601F1D1300083B1B685A10C7
:100B00008A70D2B23B49D2005B0055589B0A039AC7
:100B10009B009560ED18029B069A043B1B685B10D6
:100B20009B00D3180293314B1B78002B00D02CE58F
:100B30002B68019A1C1213402B4A9B009B580435CA
:100B400005E53B1F1868FFF71BFCA40006003F1BD0
:100B50001E2827DC00280DDC244B1B78002B00D03E
:100B600013E52B68019A1C1213401F4A9B009B58E7
:100B70000435ECE401F08AF9033E361801F086F9F9
:100B80001D4B801B9842F9D8184B1B78002B00D0C6
:100B9000FBE42B68019A1C121340134A9B009B58DC
:100BA0000435D4E40123039A137001F06FF9039B19
:100BB0000A3886195E60FBE43B1F1868FFF7E0FB0C
:100BC000A40006003F1B002818DC084B1B78002BF4
:100BD00000D0DAE42B68019A1C121340024A9B00F1
:100BE0009B580435B3E4C046189900005404002013
:100BF000489B0000B41C00209F860100C64B984211
:100C000003DD1D22C54B1A70BFE40123039A137044
:100C100001F03CF9FA239B005E43039B0A3E301827
:100C20005860C5E4A300FF1A002320001A00390011
:100C3000FFF7DCFBBA4EBB4C3168200002F0D0FE5F
:100C40003168200003F01BF83168200001F0EAFB56
:100C5000B24B1B78002B00D097E42B68019A1C1232
:100C60001340B14A9B009B58043570E4AB4BA40081
:100C70001B783F1B002B00D087E42B68019A1C12C5
:100C80001340A94A9B009B58043560E4039802F086
:100C900023FDA24B1B78002B00D076E42B68019A31
:100CA0001C121340A04A9B009B5804354FE43B1F85
:100CB0001868002838D1083B1868C3071ED54010B3
:100CC0003A0001234100083A0B431360002859DD24
:100CD00001234200391F1A430A603A00083A126899
:100CE0001A41101A3A000C3A116819421FD0C01864
:100CF0009840A4001843029BE05027E083070FD1DF
:100D000004280DD90F2302681340062B02D1FFF7E8
:100D100043FBD5E7052B03D1FFF73EFB8000CFE770
:100D200019227E4B1A7030E440100138CEE78A0752
:100D300023D1042921D90F220E683240062A15D169
:100D4000013080004358029AA400A350734B1B78D3
:100D5000002B01D0FFF719FC2B68019A1C121340DD
:100D6000714A9B009B580435FFF7F1FB052A04D11B
:100D700008180079A4004000BCE71922674B1A70DC
:100D8000FFF703FC0435E1E7A300069AFB189B1A62
:100D9000D82B13DC0122631E002C14DC5F4B1B7864
:100DA000002B01D0FFF7F1FB2B68019A1C121340B6
:100DB0005D4A9B009B580435FFF7C9FB1A22574B2D
:100DC0001A70FFF7E2FB3A601C000437E3E7069A6B
:100DD0003B1D9B1A514ED82B03DD1A233370FFF7AE
:100DE000D4FB069B029AA40093422AD23B1F1868A8
:100DF000FFF7C6FA011E21DD029B0C3B1A68521058
:100E000082421BDB9007801A484B4018C018029B97
:100E10008000C2583B1B1A60404B3F1B1B780437B5
:100E2000002B01D0FFF7B1FB2B68019A1C12134075
:100E30003D4A9B009B580435FFF789FB2023337004
:100E4000EAE71823FBE7A3009C46FE1A002C17DCF8
:100E50001C22324B1A70002333606346FF1A2F4B5B
:100E600004371B78002B01D0FFF78FFB2B68019A0A
:100E70001C1213402C4A9B009B580435FFF767FB5C
:100E8000002033685A108300F15801230B4003D12E
:100E90000D21224A1170DFE749108A4200DD0A0065
:100EA00001308442EFDC012352001343D4E7A30056
:100EB0009C46FE1A002C17DC1C22184B1A700023CB
:100EC00033606346FF1A154B04371B78002B01D0A3
:100ED000FFF75BFB2B68019A1C121340124A9B0020
:100EE0009B580435FFF733FB002033685A1083000A
:100EF000F15801230B4003D10D21084A1170DFE79F
:100F000049108A4200DA0A0001308442EFDC0123F2
:100F100052001343D4E7C04680EE3600540400204C
:100F2000780700205504002018990000FCFFFF3FBF
:100F30003B00083B1868FFF723FA3B1F06001868C0
:100F4000FFF71EFA0023864200DA0433A4003A1B9E
:100F500017001360E34B04371B78002B01D0FFF719
:100F600014FB2B68019A1C121340DF4A9B009B580C
:100F70000435FFF7ECFA3B00083B1868FFF700FA6E
:100F80003B1F06001868FFF7FBF9F30FC217B042CA
:100F90005341A4003A1B17009B001360D14B043748
:100FA0001B78002B01D0FFF7F0FA2B68019A1C1276
:100FB0001340CD4A9B009B580435FFF7C8FA3B000D
:100FC000083B18683B1F1968A600BE1B042381421A
:100FD00002D0042802D8002333601CE00123184209
:100FE00001D01942F7D103239C461842F3D102687D
:100FF0000C331A40042AEED162461142EBD1042987
:10100000E9D90A681340042BE5D1FFF7D0F9431E54
:10101000984180003060B34BA4001B783F1B04371D
:10102000002B01D0FFF7B1FA2B68019A1C12134074
:10103000AD4A9B009B580435FFF789FA3B00083BFB
:1010400018683B1F1968A600BE1B0023814202D00E
:10105000042802D8042333601CE00123184201D085
:101060001942F7D103239C461842F3D102680C338E
:101070001A40042AEED162461142EBD10429E9D983
:101080000A681340042BE5D1FFF791F94342584118
:1010900080003060934BA4001B783F1B0437002B6B
:1010A00001D0FFF772FA2B68019A1C1213408E4A86
:1010B0009B009B580435FFF74AFA3B00083B186831
:1010C000FFF75EF93B1F06001868FFF759F9F317A1
:1010D000C20F86425341A4003A1B17009B001360C5
:1010E000804B04371B78002B01D0FFF74EFA2B689A
:1010F000019A1C1213407C4A9B009B580435FFF751
:1011000026FA3B00083B1868FFF73AF93B1F060038
:101110001868FFF735F90023864200DD0433A40088
:101120003A1B170013606F4B04371B78002B01D05C
:10113000FFF72BFA2B68019A1C1213406A4A9B0096
:101140009B580435FFF703FA3B1F1B68A400043BC0
:101150005A1E93413A1B17009B001360614B0437E2
:101160001B78002B01D0FFF710FA2B68019A1C1294
:1011700013405D4A9B009B580435FFF7E8F93B009C
:10118000083B1868FFF7FCF83B1F06001868FFF7DC
:10119000F7F832180120A4003B1B1F005200024345
:1011A0001A60504B04371B78002B01D0FFF7EDF984
:1011B0002B68019A1C1213404B4A9B009B58043524
:1011C000FFF7C5F93B00083B1868FFF7D9F83B1F4C
:1011D00006001868FFF7D4F8321A0120A4003B1B60
:1011E0001F00520002431A603E4B04371B78002B4D
:1011F00001D0FFF7CAF92B68019A1C1213403A4A32
:101200009B009B580435FFF7A2F93B00083B186888
:10121000FFF7B6F83B1F06001868FFF7B1F80200A9
:101220000120A4003B1B1F007243520002431A60BE
:101230002C4B04371B78002B01D0FFF7A6F92B6845
:10124000019A1C121340284A9B009B580435FFF753
:101250007EF93B1F1868FFF793F8061E17D11F226F
:10126000204B1A70A4003B1B1F001E601D4B04374F
:101270001B78002B01D0FFF788F92B68019A1C120C
:101280001340194A9B009B580435FFF760F93B0057
:10129000083B1868FFF774F8310005F05FFA012683
:1012A00040000643DEE73B1F1868FFF769F8061E9B
:1012B0001CD11F220B4B1A70A4003B1B1F001E6089
:1012C000084B04371B78002B01D0FFF75EF92B6821
:1012D000019A1C121340044A9B009B580435FFF7E7
:1012E00036F9C04654040020189900003B00083B22
:1012F0001868FFF745F8310005F016FB0126490094
:101300000E43D9E73B1F1868FFF73AF8C217801859
:1013100050400122A4003B1B1F00400010431860F6
:10132000F14B04371B78002B01D0FFF72EF92B6807
:10133000019A1C121340ED4A9B009B580435FFF79D
:1013400006F9A300FE1A3068012C24D1FFF718F823
:101350000494079007F088FB0799002900DC01211D
:1013600005F0E2FA049BA400C918012349001943BF
:10137000DD4B3F1B1B7831600437002B01D0FFF79A
:1013800004F92B68019A1C121340D84A9B009B5801
:101390000435FFF7DCF8FEF7F3FF04907068FEF702
:1013A000EFFF049B0130C31A0793D3E7A300FE1A93
:1013B00031002000049300F073FF049B3060FF1A9B
:1013C000C94B04371B78002B01D0FFF7DEF82B68E0
:1013D000019A1C121340C54A9B009B580435FFF725
:1013E000B6F83B00083B1868FEF7CAFF3B1F060033
:1013F0001868FEF7C5FF02000120A4003B1B1F0078
:101400003240520002431A60B74B04371B78002B5E
:1014100001D0FFF7BAF82B68019A1C121340B34AA7
:101420009B009B580435FFF792F83B00083B186877
:10143000FEF7A6FF06003B1F1868FEF7A1FF32006B
:1014400002430120A4003B1B1F00520002431A600C
:10145000A54B04371B78002B01D0FFF796F82B68BB
:10146000019A1C121340A14A9B009B580435FFF7B8
:101470006EF83B00083B1868FEF782FF06003B1F32
:101480001868FEF77DFF320042400120A4003B1B9C
:101490001F00520002431A60934B04371B78002B45
:1014A00001D0FFF772F82B68019A1C1213408F4A83
:1014B0009B009B580435FFF74AF83B1F1868FEF75E
:1014C0005FFFC0430122A4003B1B1F0040001043EC
:1014D0001860854B04371B78002B01D0FFF755F8B7
:1014E0002B68019A1C121340804A9B009B580435BC
:1014F000FFF72DF83B00083B1868FEF741FF060098
:101500003B1F1868FEF73CFF320082405100012269
:10151000A4003B1B1F000A431A60734B04371B785F
:10152000002B01D0FFF731F82B68019A1C121340F1
:101530006E4A9B009B580435FFF709F83B00083BB7
:101540001868FEF71DFF06003B1F1868FEF718FF1E
:101550003200024151000122A4003B1B1F000A433C
:101560001A60614B04371B78002B01D0FFF70DF890
:101570002B68019A1C1213405C4A9B009B5804354F
:10158000FEF7E5FF3B000C3B1868FEF7F9FE3B0059
:10159000083B06001868FEF7F3FEF1170200C317B8
:1015A000300005F013FA3B1F049005911868FEF710
:1015B000E7FE02000498059905F0BCF943000120FC
:1015C000A4003E1B37001843474B30601B7804379C
:1015D000002B01D0FEF7D9FF2B68019A1C12134093
:1015E000424A9B009B580435FEF7B1FFA300FE1A48
:1015F000310020000493FEF7DFFD049B3060FF1AEA
:10160000394B04371B78002B01D0FEF7BEFF2B6847
:10161000019A1C121340354A9B009B580435FEF773
:1016200096FFA300FE1A310020000493FEF7D4FDBC
:10163000049B3060FF1A2C4B04371B78002B01D021
:10164000FEF7A3FF2B68019A1C121340274A9B0048
:101650009B580435FEF77BFFA300FF1A39002000DA
:10166000FEF7CCFD204B1B78002B01D0FEF78DFF41
:101670002B68019A1C1213401C4A9B009B5804358E
:10168000FEF765FFA300FE1A310020000493FEF769
:10169000E7FD049B3060FF1A134B04371B78002BC7
:1016A00001D0FEF772FF2B68019A1C1213400F4AFB
:1016B0009B009B580435FEF74AFFA300FF1A390030
:1016C0002000FEF703FE084B1B78002B01D0FEF72D
:1016D0005CFF2B68019A1C121340044A9B009B5824
:1016E0000435FEF734FFC04654040020189900006A
:1016F000A300FE1A310020000493FEF720FE049B95
:101700003060FF1AF14B04371B78002B01D0FEF735
:101710003CFF2B68019A1C121340ED4A9B009B581A
:101720000435FEF714FF069B3E1DF31AE74CD82B39
:1017300003DD1A232370FEF728FF00F0B1FB4300FE
:101740000120184323783860002B02D03700FEF7C1
:101750001CFF2B68019A1C121340DD4A9B009B580A
:1017600037000435FEF7F3FE069B3E1DF31AD74CF7
:10177000D82B03DD1A232370FEF707FF00F086FB4A
:10178000D44B400018400123184323783860002BC5
:1017900002D03700FEF7F9FE2B68019A1C121340A5
:1017A000CB4A9B009B5837000435FEF7D0FE01233F
:1017B000A600BE1B20001A003100FEF717FEC64C23
:1017C0002068643001F024FF002802D1043DFEF7B8
:1017D000EFFE039B21685A78C04802F05EFA0123AD
:1017E000039A3700137000F051FBBD4B22681B6851
:1017F000063253431818039B5860FEF7D9FEA60023
:10180000BE1B2000012300223100FEF7EFFDB24C89
:101810002068643001F0FCFE0028D7D0AF4802F009
:1018200037F8DCE7A4003E1BFEF758FE3700A74B55
:1018300030601B780437002B01D0FEF7A6FE2B6822
:10184000019A1C121340A24A9B009B580435FEF7D4
:101850007EFEA4003E1B300000F058FB37009B4B7F
:1018600030601B780437002B01D0FEF78EFE2B680A
:10187000019A1C121340964A9B009B580435FEF7B0
:1018800066FEA4003E1B300000F042FB37008F4B89
:1018900030601B780437002B01D0FEF776FE2B68F2
:1018A000019A1C1213408A4A9B009B580435FEF78C
:1018B0004EFEA4003E1B300000F02CFB3700834B93
:1018C00030601B780437002B01D0FEF75EFE2B68DA
:1018D000019A1C1213407E4A9B009B580435FEF768
:1018E00036FEA4003F1B380000F032FB774B1B781C
:1018F000002B01D0FEF749FE2B68019A1C12134001
:10190000734A9B009B580435FEF721FEA300FE1A84
:1019100031002000049300F03BFB049B3060FF1A71
:101920006A4B04371B78002B01D0FEF72EFE2B6884
:10193000019A1C121340664A9B009B580435FEF71F
:1019400006FEA4003F1B380000F05CFB5F4B1B78D9
:10195000002B01D0FEF719FE2B68019A1C121340D0
:101960005B4A9B009B580435FEF7F1FD01212000E6
:1019700000F030FB554B1B78002B01D0FEF705FE25
:101980002B68019A1C121340514A9B009B58043546
:10199000FEF7DDFD0021200000F01CFB4B4B1B7807
:1019A000002B01D0FEF7F1FD2B68019A1C121340A9
:1019B000474A9B009B580435FEF7C9FDA4003E1B17
:1019C000300000F03BFB3700404B30601B780437A1
:1019D000002B01D0FEF7D9FD2B68019A1C12134091
:1019E0003B4A9B009B580435FEF7B1FDA4003E1B0B
:1019F000300000F037FB3700344B30601B78043781
:101A0000002B01D0FEF7C1FD2B68019A1C12134078
:101A10002F4A9B009B580435FEF799FDA4003F1BFD
:101A2000380000F0F9FA294B1B78002B01D0FEF7A3
:101A3000ACFD2B68019A1C121340254A9B009B5851
:101A40000435FEF784FDA4003F1B380002F098FB2C
:101A50001E4B1B78002B01D0FEF797FD2B68019AD7
:101A60001C1213401A4A9B009B580435FEF76FFD69
:101A7000A4003E1B300002F02BFC3700134B3060FB
:101A80001B780437002B01D0FEF77FFD2B68019AED
:101A90001C1213400E4A9B009B580435FEF757FD5D
:101AA000A4003F1B380002F03BFB084B1B78002BC7
:101AB00001D0FEF76AFD2B68019A1C121340044AFC
:101AC0009B009B580435FEF742FDC046540400209D
:101AD00018990000FEFFFF7F7807002055040020C2
:101AE00004000020A4003E1B300002F02FFB370052
:101AF000B14B30601B780437002B01D0FEF745FD59
:101B00002B68019A1C121340AC4A9B009B58043569
:101B1000FEF71DFDA300FF1A3900200000F0F6FEBD
:101B2000A54B1B78002B01D0FEF72FFD2B68019AE7
:101B30001C121340A14A9B009B580435FEF707FD79
:101B4000A300FF1A3900200000F06AFD9A4B1B78B1
:101B5000002B01D0FEF719FD2B68019A1C121340CF
:101B6000964A9B009B580435FEF7F1FCA300FF1A30
:101B70003900200000F064FD8F4B1B78002B01D052
:101B8000FEF703FD2B68019A1C1213408B4A9B0041
:101B90009B580435FEF7DBFCA300FF1A3900200038
:101BA00000F076FD844B1B78002B01D0FEF7EDFC96
:101BB0002B68019A1C121340804A9B009B580435E5
:101BC000FEF7C5FCA300FE1A31002000049302F0CA
:101BD000C1FB049B3060FF1A774B04371B78002B46
:101BE00001D0FEF7D2FC2B68019A1C121340734AF5
:101BF0009B009B580435FEF7AAFCA300FE1A310097
:101C00002000049302F0BEFB049B3060FF1A6A4B75
:101C100004371B78002B01D0FEF7B7FC2B68019A24
:101C20001C121340654A9B009B580435FEF78FFC3D
:101C3000A300FE1A31002000049302F064FB049B11
:101C40003060FF1A5C4B04371B78002B01D0FEF785
:101C50009CFC2B68019A1C121340584A9B009B580D
:101C60000435FEF774FCA300FE1A31002000049333
:101C700002F062FB049B3060FF1A4F4B04371B7865
:101C8000002B01D0FEF781FC2B68019A1C12134037
:101C90004A4A9B009B580435FEF759FCA300FF1AE3
:101CA0003900200000F0D4FD434B1B78002B01D0FD
:101CB000FEF76BFC2B68019A1C1213403F4A9B00F5
:101CC0009B580435FEF743FCA300FF1A390020009F
:101CD00000F006FD384B1B78002B01D0FEF755FCB9
:101CE0002B68019A1C121340344A9B009B58043500
:101CF000FEF72DFCA300FE1A31002000049300F033
:101D00001BFE049B3060FF1A2B4B04371B78002B03
:101D100001D0FEF73AFC2B68019A1C121340274AA7
:101D20009B009B580435FEF712FCA300FF1A3900F4
:101D3000200000F075FD204B1B78002B01D0FEF732
:101D400024FC2B68019A1C1213401C4A9B009B58D0
:101D50000435FEF7FCFBA300FF1A3900200001F058
:101D6000DDFB154B1B78002B01D0FEF70EFC2B681A
:101D7000019A1C121340114A9B009B580435FEF730
:101D8000E6FBA300FE1A31002000049301F0C6FB1D
:101D9000049B3060FF1A084B04371B78002B01D0DE
:101DA000FEF7F3FB2B68019A1C121340034A9B00B9
:101DB0009B580435FEF7CBFB540400201899000013
:101DC0000023F7B55A1E0192002B07DA00F0E8FD58
:101DD00001F060FE01F086FF6423019300263000CD
:101DE000194B1968B14212DD184B1A6801328A4248
:101DF0000FDAF0241A601D68154F6C43E35D002B69
:101E00001FD0E419022B06D12000FEF77FFB019BB7
:101E1000D8E70022EDE7012B0DD1002801D100F019
:101E200035F8F0226A43BB185B680A49C31A8B4233
:101E300001D80223BB54F0235D43054BEB5C022B1E
:101E4000E2D00136CCE7C0467C070020000000202D
:101E5000541300209F860100002070470020704727
:101E6000002070470020704701220020054B0649E2
:101E70001A615850043103305850083180185850B6
:101E80001A60704700800040040500000122034BE7
:101E90001A64A822D20098587047C04600800040BB
:101EA00010B5FFF7F3FFFA21890004F0CDFB10BD58
:101EB00010B50100014802F07CFD10BDDC120020CD
:101EC00000487047789B00001A20704770B5054E97
:101ED0000400335C0D008B4202D003F09BF93555B2
:101EE00070BDC0468007002070B50024064D635DBC
:101EF000012B05D10021200003F08CF9002363554C
:101F000001341A2CF2D170BD800700200D207047DB
:101F100035207047036870B55B100120052B12D87F
:101F2000094A9B009C58094D2B5D002B05D00021D0
:101F3000200003F06FF900232B55200003F018F860
:101F400043000120184370BD609B00008007002003
:101F5000036870B55D10192D14D80B4E4468735D7D
:101F6000012B05D00121280003F054F901237355FA
:101F7000064964108C4202DCE143C9172140280065
:101F800003F07CF870BDC04680070020FF0300000E
:101F90000B6870B55D10192D16D80024012804DDDA
:101FA0004C68043C63425C416400094E735DA3428B
:101FB00004D02100280003F02DF97455280003F007
:101FC0005DF90423012800D00023180070BDC0462D
:101FD0008007002070B504000D0019280ED8084EA7
:101FE000335C012B04D0012103F014F90123335594
:101FF000290020004D1EA94103F02AF970BDC046FA
:102000008007002010B543680068191F4B425941F2
:102010004010FFF7DFFF10BD37B569460A00064BD9
:1020200030CB30C203680220042B02D100F008FB41
:1020300037BD00F02DFBFBE7589B000010B5084CA6
:10204000237D002B05D00021142003F0E3F80023AA
:102050002375142003F012F943425841800010BD4B
:102060008007002010B5084CA37D002B05D000216F
:10207000162003F0CFF80023A375162003F0FEF816
:1020800043425841800010BD8007002070477047D0
:1020900010B5034A0421034801F02CFA10BDC046D4
:1020A0000800002023A10000E12110B549020948E1
:1020B00002F05CFDFFF7D8FE0A2002F053FF002378
:1020C000FF21054A995401331A2BFBD100F0B4FDCE
:1020D00010BDC046DC12002080070020F8B50B4E72
:1020E000070030000D0002F089FD0400A84200DD69
:1020F0002C003D00EB1B9C4205DD300002F088FD0A
:1021000028700135F6E72000F8BDC046DC1200203B
:1021100010B50100014802F031FD10BDDC120020B5
:1021200010B5054C200002F037FDE12120004902E6
:1021300002F01CFD10BDC046DC120020064B012041
:102140001A68064B06491A6000239A00013388502A
:10215000642BFAD17047C046A40700209C070020DA
:10216000AC24002000B59BB00200054901A806F090
:10217000F1FC01A801F0A8FB01F0B4FDFCE7C046AA
:10218000FE9B000037B5184D04002868002801D0D8
:1021900006F0F2F8A400200006F0E4F82860002819
:1021A00002D11248FFF7DEFF01AB984207D2104B75
:1021B00002196B440193934201D20E48F2E70428BE
:1021C00002D808302860083C2B680B4A1C191360A1
:1021D0000A4B01201C60002309499A0001338850F2
:1021E000642BFAD137BDC046A4070020A49B000091
:1021F0001CFCFFFFD49B00009C070020A0070020D0
:10220000AC24002070B50D4D0D4E04004B1C286809
:102210009B003668C318B34203D90A20FEF758F969
:1022200070BD2B600500AB4205D80F2309011C408F
:1022300021430160F4E704C5F5E7C0469C07002090
:10224000A00700200322CB1C70B50C00D917114049
:10225000C9180500891000220420FFF7D3FF0023CE
:10226000A34206DBE343DB171C4000230419237160
:1022700070BDE95CC21811710133F1E710B5830735
:1022800006D1042804D90F2208C81340042B03D018
:102290000E20FEF71DF9014810BDC0460E9C00003F
:1022A00010B503240868044006D1042804D90F237C
:1022B00002681340042B03D00E20FEF709F910BD6D
:1022C000FFF7DCFF03782100233B5A4253411022E1
:1022D000C01806F00FFD80239B05C218044B9A42DC
:1022E00001D91420E9E7430001201843E7E7C0467D
:1022F000FFFFFF3F70B501240B680D001C4032D07A
:102300005C102000012404F0BDFC284904F088FB87
:1023100005F050FF02F0FAFF0022254B2D6805F072
:102320001FF9002200232C4004F046FB002822D095
:10233000002C1CD06C10200004F0A4FC1B4904F0FD
:102340006FFB05F037FF02F0E1FF0022184B05F0AC
:1023500007F90022174B04F0DFFC05F0BBFE430039
:102360000120184370BD0D20FEF7B2F8C9E70D201B
:10237000FEF7AEF8DFE7002C13D06C10200004F05D
:1023800081FC0A4904F04CFB05F014FF02F0BEFF8B
:102390000022074B05F0E4F80022064B05F052FB43
:1023A000DBE70D20FEF794F8E8E7C046D3023739A3
:1023B0000000D0400000E03F10B5034A022103486E
:1023C00001F098F810BDC046280000200F9C0000C6
:1023D0000020704710B51E20FEF77AF810BD10B52A
:1023E0001E20FEF775F810BD10B51E20FEF770F820
:1023F00010BD10B51E20FEF76BF810BD10B51E20E5
:10240000FEF766F810BD10B51E20FEF761F810BD8E
:1024100010B51E20FEF75CF810BD10B51E20FEF7AB
:1024200057F810BD7047000010B5034A0921034852
:1024300001F060F810BDC04638000020219C00006B
:102440000120034B1860034B1B68834018437047FF
:10245000BC070020A8070020F0B5EFF3108101238E
:10246000194083F31088134C134AA4461268134E84
:10247000013A9340124F134A002B17D014680342BD
:102480000FD03D682C60C046C046C046C046C0461E
:10249000C046C046C0460C4C1568246825605B08E1
:1024A000EAE765462C6014683460F8E781F3108829
:1024B000F0BDC04608050050C80000200C050050C3
:1024C000C8070020C4070020C007002030B585B031
:1024D00001AD0C220649280005F058FF0024285DB4
:1024E00001210134FFF7F2FC0C2CF8D105B030BD0E
:1024F000AD9C0000F0B585B06A463C4B3C4913806A
:102500000F2301AF93700C310922380005F03EFF14
:10251000FFF7C6FC374B384DC0182B68984201D2E4
:1025200000232B602C68002C44D13E5D012130003B
:10253000FFF7CCFC01340121300002F089FE092CA8
:10254000F3D100246B461E5D01213000FFF7BEFC75
:1025500001340021300002F07BFE032CF2D1C820B0
:1025600080000138C046C046C046C046C046C0468E
:10257000C046C046C046C046C046C046F1D1002154
:102580000520FFF7A3FC6B4600211878FFF79EFC9F
:102590006B4600215878FFF799FC6B46002198782C
:1025A000FFF794FCFFF77CFC002413302860200028
:1025B00005B0F0BDFFF774FC2B6800249842F6D3F9
:1025C000052002F0D5FC0D4B0D4EC0180BD4306029
:1025D0003068032104F0C2F800230A4A30602B60FF
:1025E00013600124E3E73460F2E7C0460D0E0000FB
:1025F000AD9C000010270000B4070020C8FEFFFFBC
:10260000A8070020BC07002010B50124044002D018
:102610004410200010BD0D20FDF75AFFF9E700001F
:102620000022054B10B51A60044B1B68934201D081
:1026300001F01EFF002010BDB8070020001200208E
:1026400070B508680D00FFF7DFFF04006868FFF74A
:10265000DBFF621E0100042A14D8451E042D11D888
:1026600005236B439B18012215009D402B00064853
:1026700005682B430360054B1B68002B02D020002C
:1026800001F0F7FE002070BDB80700200012002006
:1026900070B508680D00FFF7B7FF04006868FFF722
:1026A000B3FF621E0100042A13D8451E042D10D862
:1026B00005236B439B1801229A4007480368934304
:1026C0000360064B1B68002B03D00022200001F0A2
:1026D000D0FE002070BDC046B807002000120020C8
:1026E000F0B5050089B008680C00FFF78DFF069073
:1026F000022D36DD6068FFF787FF0190A068FFF7C5
:1027000083FF04000127231D661E0793731C029399
:10271000079B9E4235D0052373430593019B019D82
:1027200005330493049BAB421ED0042E16D86B1EB7
:10273000042B13D80122059B2349013B5B199A40C6
:102740009446224A0B681068069A3A4003920DD0CC
:1027500062461A430A60012200280DD17F0001352C
:10276000E0E701240194CDE7029ECFE76246934360
:102770000B600028F2D0039A0299280001F079FE3C
:10278000ECE7019B1E1D042E1AD8012C18D1002540
:1027900005273B0021006B439B1999400B000A4A17
:1027A000013511689943094B11601B68002B05D056
:1027B000019B0022581D290001F05BFE052DE8D188
:1027C000002009B0F0BDC046B8070020001200206C
:1027D00010B5041E10DA1A240A4BA400E258012393
:1027E0009340094A09491360094A1160094A0A4994
:1027F00011600A4A136010BDFFF766FBA042EADDD4
:10280000EAE7C046B4A30000C40700200805005052
:10281000C8070020C00700200C0500501805005014
:102820000200086810B5C3070DD540101823012A0F
:1028300003DD4A68042A00D10833044A1360FFF715
:10284000C7FF002010BD01204042EFE7C800002074
:102850002B4BF7B51B680C00002B03D10120404225
:10286000FFF7B6FF0126246834421AD0FF22631016
:10287000120260121040DAB21043FF221B0212044F
:10288000134018431F4B1B68202B06D1B4401E4B2E
:10289000A40EA400E35800021843FFF7DDFD00205A
:1028A000FEBD03252540FAD1042CF8D90F23226858
:1028B0001340062BF3D1FF27130901933F02019B1D
:1028C0009D42ECDA0135AB00E3583342F7D05A10A1
:1028D0005812D1B238400843FF21120209040A40BD
:1028E0001043084A1268202A06D15B009B0E064955
:1028F0009B00020258581043FFF7AEFDDFE7C046C9
:10290000C4070020C8000020A09E0000086810B581
:10291000C30703D5FFF778FE054B1860054B1B680E
:10292000002B03D0024B186801F0A4FD002010BD5D
:10293000B8070020001200200868F8B5C3071AD5B0
:10294000FFF762FE0300203B5E2B25D80520012205
:1029500058430023114E451DA84219D005211024CB
:10296000375C3C4200D09B180139520064100029AA
:10297000F7D10130F0E783070ED104280CD90F22DC
:1029800003681A40042A07D11B0905D00079D9E74A
:1029900001205B001843F8BD0120FCE7C29C000049
:1029A0007FB5A04C2368002B0AD19F4A1268002AE9
:1029B00006D19E4B1B68002B01D0FFF79BFD7FBD0E
:1029C0009B4D2A68002A26D1984A1268002A1BD0FB
:1029D000FFF790FD0028F2D0FFF778FD924B2468B6
:1029E0001A681C60002A16D0002C14D101AD0C22EC
:1029F0009049280005F0CAFC285D00210134FFF74A
:102A000065FA0C2CF8D1DAE7874A1268002AE5D17A
:102A1000002BE3D0E0E700210D2002F019FC00219B
:102A20000E2002F015FC00210F2002F011FC2E6890
:102A3000012E5DD0022E00D1A2E0002E51D1013630
:102A40003100794C04202368994302F001FC0421F1
:102A50002368052019404B42594102F0F9FB10212F
:102A60002368062019404B42594102F0F1FB8021B6
:102A70002368090119404B4259410C2002F0E8FB40
:102A800080212368090219404B4259410B2002F072
:102A9000DFFB80212368490219404B4259410A203B
:102AA00002F0D6FB80212368890219404B4259412C
:102AB000092002F0CDFB80212368C90219404B4256
:102AC0005941082002F0C4FB802321681B031940F0
:102AD0004B425941072002F0BBFB31000D2002F0B0
:102AE000B7FB2B680321581C03F01EFF296066E723
:102AF00002214D4C0720236819404B42594102F0F6
:102B0000A7FB0820216801404B42594102F0A0FB7D
:102B100080212368C90019404B425941052002F029
:102B200097FB80212368490119404B4259410620F7
:102B300002F08EFB80212368C90119404B425941A4
:102B4000042002F085FB80212368890319404B4251
:102B500059410A2002F07CFB802321681B041940A4
:102B60004B425941092002F073FB31000C2002F066
:102B70006FFB31000B2002F06BFB31000E20AEE743
:102B80002021294C0720236819404B42594102F06B
:102B90005FFB40212368082019404B42594102F055
:102BA00057FB80212368092019404B42594102F00C
:102BB0004FFB80212368490019404B4259410A20AC
:102BC00002F046FB80212368890019404B4259419D
:102BD0000B2002F03DFB80212368890119404B4204
:102BE00059410C2002F034FB80212368490319402D
:102BF0004B425941062002F02BFB80212368C90378
:102C000019404B425941042002F022FB80232168E5
:102C10005B0419404B425941052002F019FB012188
:102C20000F205CE7B8070020B0070020BC07002099
:102C3000AC070020AD9C0000012010B54042FFF71A
:102C4000C7FD0020FFF708FC10BD000010B5034AC7
:102C50000921034800F04EFC10BDC0468000002052
:102C6000A09F000030B502248025094B094AED00E1
:102C70009C505C59002CFCD0A124E400884202D373
:102C80000021995030BD8025ED0018514019F5E71D
:102C900000E001400405000010B5002806D1C02066
:102CA000B02140028902FFF7DDFF10BDB020802176
:102CB0008002C902F7E7000043425841064B4042F8
:102CC0001840B0239B02C018036800201A0E532A34
:102CD00001D11B02180A704700C0FEFF30B5012465
:102CE0008025054B054AED009C505C59002CFCD01A
:102CF00001600021995030BD00E001400405000052
:102D000043425841074B40421840B0239B02C01831
:102D1000A62310B50902DB05090A1943FFF7DEFFF8
:102D200010BDC04600C0FEFF70B5012480250D4BCC
:102D30000D4EED009C515C59002CFCD0002902DCAA
:102D400000229A5170BD557814782D02254394784D
:102D5000013924042543D478043224062C4310C0BE
:102D6000ECE7C04600E001400405000070B5050036
:102D70004B680A009C1C2100A400FFF7D5FF28190E
:102D800070BD0000134B1B68002B0CD08022B023B9
:102D9000D2029B0200280BD11A1D5B681B0E522B1E
:102DA00000D110007047B022C02392025B02F1E70D
:102DB00082420DD903681B0E522B09D1436802339E
:102DC0009B00C018824203D903681B0E522BE9D026
:102DD0000020E7E7CC08002070B50020FFF7D2FF05
:102DE000FF260500002801D1280070BD03681C14CF
:102DF0003440FFF7C7FFDA2CF4D10500F2E70000FA
:102E00008022F0B55200A1B00021674805F0C7FA52
:102E1000802200215200654805F0C1FA644BFF276B
:102E20001B681A00049353425A4110000592FFF7A1
:102E300033FF049C0020631E9C415E4B64421C4097
:102E40005D4BE418FFF7C8FF0600002E2DD1049853
:102E5000FFF732FF411C0598FFF752FF059A574DC7
:102E6000534B2C601A60FFF75BF9514B64201B68D1
:102E7000A0215A4253414F4A5B421340B0222C6872
:102E800092029B18E41A6043490203F067FCA022F7
:102E90005202030000924A49220007A805F05AFE98
:102EA00007A800F011FD21B0F0BD32681314121212
:102EB0003A403B4003921A000A3A092A49D83A4B51
:102EC000039A995C002931D110223E4805F067FA37
:102ED00035002B6803991A123A40914209D11A140D
:102EE0003A400B2A27D0132A2DD00A2A01D1354B7C
:102EF0001D602800FFF746FF051EEAD1314B196817
:102F000000290FD02000FFF731FF04002D4B5B1983
:102F10005968002903D02000FFF728FF040004357A
:102F20000C2DF3D1204B0121039A99543000FFF767
:102F300029FF060089E73B40022BDADC214A9B008F
:102F4000D3185D60D5E7102200211E4805F027FA4E
:102F5000CFE71A00153A082AE8D8144A0399525CB8
:102F6000002AE3D13500152B00D01500300003688E
:102F70001A143A40152A0FD01D2A00D10025FFF758
:102F800001FF0028F3D1002D04D020002900FFF715
:102F9000EDFE0400054BC6E7039A1B123B409A4224
:102FA000EDD10500EBE7C046CC070020D408002097
:102FB000CC08002000C0FEFF04C00200D0080020A2
:102FC0003AA000003C260020F0B50020B7B0002455
:102FD000FFF7D8FE270005002600002D2ED1284D32
:102FE0002868FFF769FE32003B00019000942549F4
:102FF00004A805F0AFFD04A800F066FC224B642095
:103000001C682B68A0215A425341204A5B4213405E
:10301000B02292029B18E41A6043490203F09EFB1F
:10302000A0225202030000921949220004A805F0D0
:1030300091FD04A800F048FC37B0F0BDFF226B689A
:1030400029689C460233FF180B12013613409C423C
:1030500000DA1C00FF200A1402400392624601407D
:1030600001920091039A0B4904A805F073FD04A88E
:1030700000F02AFC2800FFF785FE0500ADE7C046FA
:10308000CC080020ADA00000D008002000C0FEFF4A
:1030900055A0000099A0000070B50020FFF70CFEBD
:1030A00004000120FFF708FE844200DA04000A4B06
:1030B0001D686A42554128001D60FFF7EDFDA02202
:1030C0006B4252021340054A28009B18044A611CB7
:1030D0001360FFF715FE70BDCC08002004800100CE
:1030E000D0080020F8B50020FFF7E6FD070001201A
:1030F000FFF7E2FD3E00224D0643224C0DD1802118
:10310000C020C9024002FFF7ADFD01213000FFF7EA
:10311000F7FD1D4B2E60236022E0874209DD00236E
:10312000B0212B60184B8902236023680020012501
:103130001CE0012380212B60144BC9022360F4E7BB
:10314000120E522A0DD0002800D02360104C1149D5
:10315000200005F029FD2000FEF7AAFEFFF79CFFE6
:10316000F8BD28005A68023292009B188B4205D2A3
:103170001A68561CE4D10028F2D0CCE72160EFE7B2
:10318000CC080020D00800200480010004C0020008
:103190008826002070A00000F0B585B003920322BD
:1031A0000333DC172C4D1440E4182B682B4F5A4284
:1031B000534180225B42D202A4103B409B18A21CC8
:1031C0000291274E910000910190316800980A18F1
:1031D00093421AD2FFF714FE2B685A4253418022C1
:1031E0005B421F40D202BF183368009A9B189F426F
:1031F0000BD21C4C1C49200005F0D6FC2000FEF729
:1032000057FE0025280005B0F0BD029B3568190661
:103210006B461A7BA423DB051343FF222F00090C06
:103220001943019B12041B04134019432800FFF7A4
:1032300055FD0837281D21003760FFF74FFD002C92
:1032400004D00A9A21003800FFF76EFD009B083B6E
:10325000FF183760D6E7C046CC08002000C0FEFF4C
:10326000D00800208826002013A0000010B5FFF72A
:10327000C7FD10BD70B59AB0FFF734FFFF22254C93
:10328000D2000021200005F08AF80020FEF7D6FECB
:1032900004280ED10020FEF7E5FE042809D1FFF72F
:1032A000FBFE1D4800F010FB1C4800F00DFB1AB09F
:1032B00070BD0020FFF790FDFF25002600280ED1ED
:1032C0000200C300E3580130591E8B41D218FF2879
:1032D000F7D1134901A805F03DFC01A8E2E7036816
:1032E0001A142A400A2A0AD11A122A40FF2A03D0A5
:1032F000D200A1180B71A050FFF744FDDEE7132A9E
:10330000FAD11B122B40FF2BF6D0DB00E21816710E
:10331000E650F1E7B41C0020E2A00000F2A000009B
:10332000FAA0000000207047012070470048704755
:10333000642600200048704733F8FFFF10B50449A9
:10334000044805F031FC24230348036010BDC04647
:1033500014A10000502600204C26002000207047B9
:103360000020704700207047002070470020704701
:1033700000207047002070470020704700207047F1
:1033800010B5034A0E21034800F0B4F810BDC04642
:10339000CC0000200EA10000044A05491368C8545F
:1033A00001339B059B0D13607047C046EC0D002058
:1033B000EC09002070B5114C114A2368834202DCED
:1033C0000023236016E0155C411C2E00FA3E012EFE
:1033D00005D899420FDA555C013D1F2D01D908002F
:1033E000ECE70100151A565C6E5401318B42FADC91
:1033F000181A206070BD1570FAE7C046F811002059
:10340000F80D002010B5FEF741FD064B1A68824208
:1034100001D900221A601B68C31A034898428041F0
:10342000404210BDE8090020204E000010B5094CB4
:10343000094A23681268934200D110BD074AD05C44
:10344000FEF766FE0028F8D0236801339B059B0D2C
:103450002360ECE7F00D0020EC0D0020EC090020CB
:1034600010B50400064B074A1B6812689B1ADB4321
:103470009B059B0DA34200DB10BDFFF7D7FFF1E7D3
:10348000EC0D0020F00D0020F7B505005668019105
:10349000B000441C06301700FFF7E2FFFB20FFF7E7
:1034A0007BFF1C20FFF778FFE8B2FFF775FFE0B263
:1034B0002412FFF771FFE0B2FFF76EFF6B46187939
:1034C000FFF76AFF0025AE4200DCF7BDAB00FB183A
:1034D0009C680135E0B2FFF75FFF2012C0B2FFF732
:1034E0005BFF2014C0B2FFF757FF200EFFF754FF19
:1034F000E9E7000070B5074E3368092B08DC0C259E
:103500005D43054C0133285164196160A26033604A
:1035100070BDC046F40D0020EC260020F0B587B049
:1035200002900C00012803DC1B20FCF7D1FF45E0D2
:10353000244B08680093830709D1042807D90F2377
:1035400002681340042B02D1FEF798FE00901D4B39
:1035500060680193830709D1042807D90F23026803
:103560001340042B02D1FEF789FE01900027164B71
:103570001B680493049BBB42D6DD0C267E43134B91
:103580000099F618306805F005FB051E05D1736833
:10359000B6680593059B9D4201DB0137EAE7306879
:1035A0000199039605F0F6FA0836002808D12100A3
:1035B0000298039B083102385B68984707B0F0BD5A
:1035C0000135E7E70E9C0000F40D0020EC260020FA
:1035D00010B5FFF73BFBFEF75BFDFEF7EDFEFEF7D8
:1035E00023FFFFF7CDFE00F0BFFD00F045FF10BD4B
:1035F000962210B512010021034804F0D0FE0022EB
:10360000024B1A6010BDC046541300207C070020F6
:10361000064B074A1B6812689B1ADB439B059B0DF0
:103620000122834200DC002210007047EC0D0020D4
:10363000F00D0020F8B505000C0016001F1E0ED17D
:103640000320FFF7E5FF002808D0FA20FFF7A4FECB
:10365000E8B2FFF7A1FEE0B2FFF79EFEF8BD501DF5
:10366000FFF7D6FF0028F9D0FB20FFF795FEE8B260
:10367000FFF792FEE0B2FFF78FFEF0B2FFF78CFE8D
:103680003012C0B2FFF788FE3C00E31B9E42E5DD2E
:103690002078FFF781FE0134F7E7000070B50024C1
:1036A000F0250B4B1B68A34202DCFFF7A1FF70BDA6
:1036B0002B006343074A9B181A78002A05D05978D3
:1036C000002311201A00FFF7B5FF0134E9E7C046D7
:1036D0007C07002054130020F8B507000024F025D3
:1036E0002B0063430C4A01349E18B74211D0317845
:1036F00000290BD00133D15C002311201A00FFF701
:1037000099FF2A000021300004F049FE0A2CE7D17D
:10371000F8BD024B1C60F9E7541300207C07002021
:10372000F3B50400100001220300FFB00D001340A8
:1037300013D002AB1A70431002AA02A953704212AE
:103740001B0E8A700B7105220B004014C8702900F3
:103750002000FFF76FFF7FB0F3BD032606401ED1A8
:1037600004281CD90F2201680A40042A29D1022307
:1037700002AA1370FEF782FD070005F01DFAF82378
:10378000FF33984200D91800B04202DC421C02AB61
:10379000DDE70136731EFB5C02AA9355F4E70428AB
:1037A00001D0002809D1032302AA04381370424231
:1037B000504102AB58700222C9E7002ECBD1042839
:1037C000C9D90F2102681140052913D1013902AE70
:1037D0003170F8211209FF3192008A4200DD0A009F
:1037E000934201DB0132D2E70133C118C97802AE3E
:1037F000F154F5E70629AED101390E0012095643FE
:103800000196F826019FFF36B742A4DC02AE317064
:103810000136934201DB019AE4E701270133990065
:10382000415839420BD03941012737700F1271705E
:10383000B7700F14090EF77031710536E9E70149C9
:10384000F2E7C04619FCFFFF70B502000024F0212A
:103850000D4E0800604380194578954203D001342D
:103860000A2CF6D170BDF022002104F098FD074A21
:103870001368013BA34200D11460002329001A0001
:103880001120FFF7D7FEEDE7541300207C0700203E
:1038900010B5B2B002236A460400137005F08CF92B
:1038A000C72800D9C7200023984207DC421C6B467A
:1038B000FE211420FFF7BEFE32B010BD6946013371
:1038C0005A1EA25CCA54EFE730B5B3B002236A4671
:1038D0000500137005F070F90400C72800D9C7244B
:1038E00000239C420BDC20003230FFF7B9FD621C44
:1038F0006B46FF211420FFF79DFE33B030BD6946B3
:1039000001335A1EAA5CCA54EBE70000F7B5234BFB
:1039100006001B68F02100930023009A9A4211DCF4
:103920000024F0231A006243019201991C4A5518A1
:103930002F78002F12D001340A2CF3D11948FFF749
:10394000C3FF29E00A005A43154882185078B04254
:1039500002D11278002A1FD10133DEE7F0223900AC
:10396000280004F01CFD02230D4A0199EB6053541A
:103970000D4AF1008A58009B6E70AE70AA602F61EC
:103980006F61A34202DC054B01341C60002331004F
:103990001A001020FFF74EFEF7BDC0467C0700203E
:1039A00054130020FBA10000B41C002010B5FFF749
:1039B00075FEFF24084AE3005B429B18074AD35C6C
:1039C000043B012B03D8E043C0B2FFF79FFF013C4B
:1039D000002CEFD110BDC046FC070000B41C002035
:1039E000F7B50E00FF247F2501901C4AE300D31A8F
:1039F0001B4A9A181278062A01D0032A1DD1FF22E9
:103A0000D2009B18186883682B401C2B15D1C36803
:103A10001A002A40042A10D102692A40192A0CD11E
:103A20001B0A01339B000C30C018FEF727FC07006F
:103A300005F0C2F80023B04209D0013C002CD4D1DB
:103A4000F7BD019AF95CD25C9142F6D101339E42F6
:103A5000F7DCE043C0B2FFF759FFEEE7B41C0020EB
:103A6000FC07000070B50500FF24084AE3005B4234
:103A70009B18074AD35CAB4203D1E043C0B2FFF7C7
:103A800045FF013C002CF0D170BDC046FC07000092
:103A9000B41C0020F7B5FEF7F9F9514B1A688242C1
:103AA00001D900221A601A684E49821A8A4200D847
:103AB00083E01860FEF7F4F9071E00D101370020FB
:103AC000FEF7BCFA01900020FEF7CCFA019B0090B3
:103AD000454C464D002B14D02368002B00D07AE0D3
:103AE0002B682760002B00D171E0414B01261B7829
:103AF000002B63D10920FFF7B5FF3E4B1E703C4BF6
:103B00001E70009B002B12D02B68002B0FD1236856
:103B10002F60002B1ED0374B01261B78002B52D173
:103B20000920FFF79FFF334B1E70314B1E70236837
:103B3000002B0FD02F4E3278002A0BD19F4200D29B
:103B400027602368FB1A312B04D90720FFF78AFF6F
:103B5000012333702B68002B0FD0254E3278002ABA
:103B60000BD1BB4200D92F602B68FF1A312F04D92B
:103B70000820FFF777FF012333702368002B0CD058
:103B8000019B002B09D11B4E3378002B02D107205B
:103B9000FFF768FF0023236033702B68002B0CD0E5
:103BA000009B002B09D1124C2378002B02D1082056
:103BB000FFF758FF00232B602370F7BD0720FFF7A6
:103BC00051FF0C4B9CE70820FFF74CFFADE7009B33
:103BD000002B9CD1ABE7009A002A95D1AAE7C046FA
:103BE000E40900200F270000D4090020DC09002090
:103BF000E0090020D809002037B500240500FFF7B0
:103C00004DFD01A80194FEF707FA21002000FEF700
:103C100007FDFEF7C5FEFEF739FAFEF738FAFFF7A3
:103C20000BF8FEF761F9A54204D0FEF787FA0248C7
:103C3000FFF74AFE37BDC046ECA10000002310B5D7
:103C400001001A001120FFF7F5FC10BD07B56B4607
:103C5000197069465A7013128B701314120ECB70C0
:103C60000A716B46010005221320FFF7E3FC07BD34
:103C700010B50A0001001220FFF752FD10BD70B50B
:103C8000050008000C003230FFF7EAFB2B00220091
:103C900000211B20FFF7CEFC70BD10B50C00030007
:103CA000110014202200FFF7C5FC10BD70B50600FE
:103CB0000020FFF767F80024FF25002801D120002D
:103CC00070BD03681A142A40152A07D11B122B4015
:103CD000B34200D10400FFF755F8EEE71D2AFAD1F0
:103CE0000024F8E7F0B580279DB0FFF79FFBA94CB3
:103CF000A94D2068FF00391A4019FEF7EFF9236833
:103D00000600C3182360002B0ED11DB0F0BD206843
:103D1000391A2818FEF7E2F9236806001B182360F9
:103D2000FEF7B4F89D4B1860002EF0DC2B78FA2BD0
:103D300000D00BE12368022B07DCFFF763FB0028B0
:103D4000E3D00120FFF736FBDFE76878AC78023874
:103D5000182823D802F06EFC0D1F24282B34223E95
:103D600068226E84D6E722222222222222222222C6
:103D7000F500FF2C12D02000FFF766FD0022884BD3
:103D8000E100CA505B181A71210013001320009241
:103D9000FFF702FA02E02000FFF7B8FD0320D1E7A9
:103DA0002000FFF751FDF9E7FFF700FEF6E7FFF708
:103DB00075FC0020FFF720FF7A48FFF785FDEDE74F
:103DC000632CEBD8784BA200D25821001520FFF7C6
:103DD000A7FCE3E700242000FFF768FF061E03D1DD
:103DE0000134642CF7D1D9E7083004F0E5FE050072
:103DF0000530FFF735FBFB20FFF7CEFA1D20FFF75C
:103E0000CBFAE0B2FFF7C8FAE8B2FFF7C5FA28121A
:103E1000C0B2FFF7C1FA3700BB1B9D42E0DD387A24
:103E2000FFF7BAFA0137F7E700211D2000910B00D8
:103E30000A00ADE7FEF744F803AC5C4A6421009049
:103E40005B4B200004F054FE02232000237004F09A
:103E5000B3FE2300020000211620FFF7EBFB9DE7D5
:103E600000244F4AE300D558002D28D06B689E00EF
:103E7000701DFFF7F5FA2B000025320008332100F2
:103E80000120FFF7D7FB0020FEF77CFF2F002E005C
:103E9000002818D1002F04D03A0001212000FFF79C
:103EA000F3FA002D04D02A0002212000FFF7ECFADB
:103EB000002E04D0320000212000FFF7E5FA013483
:103EC000FF2CCED16AE7FF2103681A120A40A242F2
:103ED00009D11A140A400B2A08D10B400CD0012B2F
:103EE0000CD0022B0CD0FEF74DFFD1E7132AFAD1EC
:103EF00000252F002E00F6E70600F4E70700F2E7A2
:103F00000500F0E70024FFF7C9FB22002100009420
:103F10002300DA20FFF740F9FF222100D2002048D9
:103F200004F03DFA3AE7012C02D1FFF74DF835E7EE
:103F3000022C02D1FFF79AF930E70120FFF75CFE6F
:103F40002CE7002321001A001A2086E7FB2B00D063
:103F5000F7E62268042A00DCEFE62E79E878154BB4
:103F6000360206439E4200DDEBE6331D9A4200DC3A
:103F7000E3E6EB5CFE2B00D0E3E66B78AC78711ED9
:103F80001B2B6BD018D8012B2BD0082B3DD0701DCC
:103F9000D8E6C046F8110020F80D0020E8090020FE
:103FA000B41C0020CEA10000AC240020E5A100003C
:103FB000E0A10000F60300001D2B60D052D31E2BA1
:103FC000E5D1012CE3D10029E1DD6B79002B03D091
:103FD0001C00322B00DD322464235C43344B1C6014
:103FE000D5E7FF2CD3D02000FFF72EFC6D79314AA6
:103FF000B31E009221002A000A20FFF7CDF82E4BB5
:10400000E400E0501B191D71C1E7632CBFD86A7929
:10401000022A13D0032A1BD0012AB8D1E979AB793F
:10402000090219432B7AA4001B0419436B7A1B065F
:104030000B435B001343214AA350A8E70029A6DDE8
:10404000B11E1C48FEF7FEF81C4BA400E0509EE792
:10405000AB79A4005A1E93419B00ECE71848FFF788
:10406000BFFC94E7FF2C92D06A79022A8FD81149BD
:104070000B2000912100B31EFFF78EF887E70B009D
:10408000632900DD6323002203A893420ADCD9439D
:104090000022C917194041180A700133009021000D
:1040A0001520E9E7A918497981540132EDE7C046A6
:1040B00004000020FE0D0020B41C0020AC240020D1
:1040C000FD0D00200120704710B5064C200000F0C7
:1040D0000BFB0549200000F02FFB0122034B1A6067
:1040E00010BDC04624120020801A0600FC110020DA
:1040F00010B501210D20FDF7E9FE01210E20FDF78D
:10410000E5FE00210F20FDF7E1FE044C200000F049
:1041100027FA1021200000F03FFA10BD0412002001
:1041200010B504680D20E30703D56410FF2C03D9F4
:104130001720FCF7CDF910BDFFF7DAFFE1B2024816
:1041400000F04CFA0020F6E70412002010B5FFF74B
:10415000CFFF0021034800F041FA4300012018433B
:1041600010BDC0460412002010B5034A07210348C1
:10417000FFF7C0F910BDC0463C01002010A20000AE
:10418000F8B5012306681E4205D045681D4202D0DD
:1041900084681C4203D10D20FCF79AF9F8BD761013
:1041A0001520802EF8D86D101620FF2DF4D864103D
:1041B000FF2C01D91720EFE70B4B1B68002B01D117
:1041C000FFF782FF094FF1B2380000F04CFBE9B273
:1041D000380000F04FFAE1B2380000F04BFA380036
:1041E00000F0ACFB0020D9E7FC11002024120020D5
:1041F000F7B501242300A0421BDD0D682C4218D026
:104200001A4B25411B684C68002B01D1FFF75CFF5E
:104210000127174EE9B2300000F025FB3C420AD0DE
:104220003C413000E1B200F025FA300000F086FB9E
:1042300000231800FEBD03252540F6D1042CF4D937
:104240000F2322681340062BEFD113090193019B22
:104250009D42EADA0135AB00E1583942F7D0491006
:10426000C9B2300000F006FAF1E7C046FC110020A8
:1042700024120020144B70B51B6805000E00002BA3
:1042800001D1FFF721FF114CEDB22900200000F011
:10429000EAFAF1B2200000F0EDF90021200000F070
:1042A000EDFA002801D0404270BD01222900200013
:1042B00000F0D4FA200000F0CEF90028FAD0200057
:1042C00000F0CEF9F0E7C046FC11002024120020D7
:1042D00010B501240368234202D04168214203D172
:1042E0000D20FCF7F5F810BD5810802801D91520D5
:1042F000F7E74910FF2901D91620F2E7FFF7BAFFC7
:1043000040002043EFE710B507211820FFF7B2FF68
:104310007F2801DD0138FF3803007F3301DA7F2079
:10432000404264235B4258437F2102F017FA012385
:1043300040424000184310BD10B508211820FFF777
:1043400099FF0300C00FC018012340101530400032
:10435000184310BD10B505211820FFF78BFF7F28EB
:1043600001DD0138FF3803007F3301DA7F2040424E
:1043700064235B4258437F2102F0F0F9430001209F
:10438000184310BD10B503211820FFF773FF7F28D5
:1043900001DD0138FF3803007F3301DA7F2040421E
:1043A00064235B4258437F2102F0D8F94300012087
:1043B000184310BDF8B50123020018009A4236DDFB
:1043C0000E68334233D003244D682C402FD1042D86
:1043D0002DD90F2229680A40062A28D1144B1B68C0
:1043E000002B01D1FFF770FEEB0704D42B681C09EA
:1043F000202C00DD20247610F1B20E4E2200300079
:1044000000F02CFA0435A700EF19AF420CD03000B1
:1044100000F021F90028FAD0300000F021F9012342
:104420004000184301C5F0E7012064002043F8BDB7
:10443000FC1100202412002000207047002070474B
:104440000020704700207047002070470020704710
:104450000020704700207047002070470020704700
:1044600000207047002070470020704700207047F0
:10447000704770477047000010B5034A0E2103488B
:10448000FFF738F810BDC0467401002051A20000AB
:1044900010B5FDF709FE0648FDF774FEFFF798F822
:1044A0000448FFF711FAFEF7E5FEFFF77FFA10BDAB
:1044B000E2040000DAA2000010B5FDF781FC10BD97
:1044C00070B5002504AC24780573A94205D10A4BC8
:1044D0000A4A23210A4803F0DDFE016009499200DF
:1044E00052589B0002715B58A40083716358856029
:1044F00043710223C37170BDF2A2000057A30000F4
:1045000000A30000B4A30000037B002B04D143737D
:104510008373036101330373704700001FB501917A
:10452000A02100240068C900D2B24450012A10D052
:10453000A24209D0032A0AD0074A8350074B019AA6
:10454000C250012343501FBD02221343F4E704224B
:10455000FBE70622F9E7C0465405000024050000E9
:1045600010B50400FFF7D0FFA1222368A179D20083
:1045700099506179064A2000995021790432995066
:10458000044B19685A689B68FFF7C8FF10BDC04606
:104590000C050000181200204BB2002B0FDB80230B
:1045A0003F290FD81F290FD80F290FD807290FD857
:1045B00003290FD81B060168074A8B5070478023D8
:1045C0009B04F8E7DB04F6E71B05F4E75B05F2E77D
:1045D0009B05F0E7DB05EEE7240500000368074ACA
:1045E00099501A00FC32D1680029FCD0A321C900DF
:1045F00058580023C0B2D3607047C0461C05000065
:1046000007B58022074BD2051A6000229A60023259
:104610001A7111230E320093034905330348FFF743
:104620004FFF07BD18120020003000400412002088
:10463000F8B505000E0017000024BC4208D02B6816
:10464000315D1B6828009847002801D00134F4E749
:104650002000F8BD704710B51C3000F0D6F910BD31
:1046600010B51C3000F0C3F910BD10B51C3000F0BF
:10467000D2F910BD70B5437E0D00002B01D1002092
:1046800070BD6430040000F0CFF90028F7D120009D
:10469000290000F09DF90120F2E70000F7B5019331
:1046A000FA23002504009B0083600D4B456008330E
:1046B00003601C300F00160000F07FF9200064300A
:1046C00000F07BF9074A2761B600B35820006375F4
:1046D000019B9B009B586576A576A375FEBDC046E1
:1046E00094A30000B4A300000123A022C375837D1E
:1046F0000E49C133FF33D2059B009950437DC1332E
:10470000FF339B009950CC220169094B5204CA50D7
:1047100005220169243BCA50827D01690833CA50D1
:104720000269417D034BD1507047C0460C06000022
:10473000240500000C050000A022002310B5046928
:10474000D200A3500A4CA1420FD90A4C8C425B41C3
:1047500009495B420B40CD21C9045B180469074934
:10476000635005210369995010BDCC235B04F5E724
:10477000A086010090D00300000098FD24050000F1
:10478000F7B5040000200D000193824265D01600A9
:10479000402A00D9402627001C37380000F023F9B2
:1047A000B1232269DB00D5508022012321699200C8
:1047B0008B50A27E002A03D1226913622269136002
:1047C0000025731EAB4207D1019B002B04D0802231
:1047D0000221236992009950012223691A622369F8
:1047E000FC33DA68002A02D19A6A002AF9D09A6A60
:1047F000002A0BD1DA60A3232269DB00D1583800EC
:10480000C9B2013500F0E4F8B542DAD3019B226960
:10481000002B0FD11300FC339B6A002B0AD101330C
:10482000A376D3612369FC33DA6C002AFCD0002222
:10483000DA640AE000230121A37651611A0023699A
:10484000FC3399680029FCD09A602369FC339A6A8A
:10485000002A01D000229A62E8B2FEBD10B5012301
:10486000FFF78EFF10BD0300AC3310B504001970C4
:10487000643000F0B8F80123637610BD0023020015
:1048800070B5AC3243760D001178B1220400006996
:10489000D20081508022216992008B50226901331D
:1048A00013622269936026006436300000F0ADF890
:1048B000002812D0300000F09AF81E4B2269D05028
:1048C0002369FC331A6A002A02D19A6A002AF9D0B5
:1048D0009A6A002A01D11A62E5E723690122002DB4
:1048E0000DD11900FC31896A002908D1DA612369E8
:1048F000FC33DA6C002AFCD00022DA6407E05A614B
:104900002369FC339A68002AFCD000229A600020B8
:104910002369FC339A6A82420BD098622169064A65
:104920008B588B501800022B03D0181F431E984140
:10493000033070BD1C050000C404000010B5012147
:10494000FFF79CFF10BD000010B51323122202498F
:104950000248FFF7A3FE10BD0040004024120020D3
:10496000F7B506000D000C008B180193019B671B27
:104970009C4207D0336821781B6830009847013487
:104980000028F3D13800FEBD70B5040008000D000A
:1049900004F012F92368020029005B6820009847A0
:1049A00070BD10B50B1E02D0FFF7EEFF030018001C
:1049B00010BD10B5FFF7F5FF10BD10B54022002166
:1049C000040003F0ECFC002320002364636410BDAA
:1049D00010B53F24026C531C2340446C9C4201D010
:1049E0008154036410BD0023036443647047436C27
:1049F000026C934206D03F21C25C01330B404364FA
:104A00001000704701204042FBE7036C406C181A0D
:104A100000D540307047436C026C934201D0C05CBB
:104A2000704701204042FBE73F22036C406C01339A
:104A30001340181A43425841C0B2704703210A4834
:104A400002680A430260094802680A430260084992
:104A5000084A094B9B1A03DD043BC858D050FBDCC5
:104A600000F012F8FBF750FB24050040540500400D
:104A7000A4A800000000002014040020FEE7FEE7C8
:104A8000FEE7FEE7FEE7FEE72D4B10B51A68D2B24F
:104A9000012A0FD12B4A126812070BD12A4AE024AF
:104AA0001168F0220800104021422DD127490968E1
:104AB00011422CD01A68D2B2012A12D121490968B8
:104AC00009070ED1F020204909680140402908D18A
:104AD0001E490968014204D18020C121C005C900D6
:104AE00042501B68DBB2012B0DD1164B1B681B0714
:104AF00009D1154B1A68F0231A40A02A0FD1134A86
:104B000012681A420ED010BD3028CFD0D2E7104A1A
:104B1000104911608021104A09021160CAE7D02AA9
:104B2000F1D1ECE70D4B1A68012A04D00C4A1A6047
:104B30001A68012AFCD1C0220A4B1A60E3E7C0467A
:104B4000E00F00F0E40F00F0E80F00F0EC0F00F0D1
:104B500004050040DFFF07C0186C004000EC064071
:104B60007593000014EC06400120704710B50368EF
:104B70001322DB69984710BD70470000054B02699E
:104B8000D1500369FC331A6A002AFCD000220120AC
:104B90001A6270471C050000030010B55C331A78D8
:104BA0001F231A401E3B19009140114AD167C222AF
:104BB000042104699200A150026953600269D36024
:104BC000A02300220169DB00CA5001230169094AC0
:104BD0005B428B500169084A8B5001690C3A8B503B
:104BE000016908328B501430FFF7FDFE10BDC0463E
:104BF00004E100E00C0500001405000010B51430BD
:104C0000FFF703FF10BD10B51430FFF704FF10BD10
:104C100010B51430FFF7EBFE10BD0000030070B5B7
:104C20005E331A780469724BE25003005D331A78E0
:104C30000469704BE250030061331C7802696E4BCB
:104C4000012C00D09EE005005F352E78A225ED00F6
:104C50005651020060321578A1220669D200B55083
:104C60000269D4509623DB00994200D88CE0962349
:104C70001B01994200D88AE096235B01994200D833
:104C800088E096239B01994200D885E0E1239B01AF
:104C9000994200D882E09623DB01994200D880E057
:104CA000E123DB01994200D87DE096231B02994263
:104CB00000D87AE0E1231B02994200D877E09623DE
:104CC0005B02994200D874E0E1235B02994200D86C
:104CD00071E0E1239B02994200D86EE0474B994274
:104CE00000D86CE0E123DB02994200D86AE0E122BF
:104CF000002312038A425B41414A5B4213408022F7
:104D000052059B1801693F4A8B50A0230422016978
:104D1000DB00CA5000210369FC33D9600369FC330E
:104D20001962012301690B6001698B60C12104696B
:104D3000890062501F215C3002780A409340623142
:104D4000314AFF3153500021415600293CDA0F23EC
:104D50000B40083B2D4C9B089B001B190324214052
:104D6000A140FC348C40DD69A5432C00C0258D405A
:104D700029002143D9611F23017819401E3B8B4034
:104D8000136070BD00246CE79E23DB02BAE79D230D
:104D90001B03B7E71E4BB5E71E4BB3E7EC239B03A2
:104DA000B0E71D4BAEE71D4BACE71D4BAAE71D4B13
:104DB000A8E71D4BA6E71D4BA4E71D4BA2E78023E8
:104DC000DB049FE71B4B9DE78C080F4BA400E41806
:104DD00003230B40FF21C025DB009940AD0066593D
:104DE0008E433100C0269E4033000B436351C2E71F
:104DF0000C050000140500006C05000090D00300B5
:104E000000D0BEFE2405000000E100E000ED00E05F
:104E100000B013000050270000A04E0000F0750005
:104E200000509D0000F0EB0000903A0100E0D70137
:104E300000B0AF0300705F07F7B5009308AB1B78B5
:104E400000250193FA2304009B0083600E4B45600C
:104E50000833036014300F001600FFF7AEFD230087
:104E60005C3327611E70009B084A9B009958230001
:104E70005D331970019B20009B009A5823005E331C
:104E8000DD701A70FEBDC04630A40000B4A300005F
:104E9000036910B51A00FC32D2680400002A0AD057
:104EA000A322D20099581430C9B2FFF791FD002215
:104EB0002369FC33DA6010BD10B50248FFF7E8FF44
:104EC00010BDC046DC1200201D2307B5022200934E
:104ED000024901330248FFF7AFFF07BD0020004041
:104EE000DC1200207047000010B500F011F8FFF749
:104EF000F9FF012000F0ECF9FFF7CAFAFFF7DCFA3E
:104F0000024B002BFAD000E000BFF7E700000000E2
:104F1000C420114B80001A5810491140C0221202BF
:104F20000A431A50C0218022490092025A501A6046
:104F30008023A3220021DB05D20099500122F93001
:104F40009A60074BFF301950C12002318000195080
:104F5000403019501A60704700E100E0FF00FFFF89
:104F600000100140014B18607047C0462C02002021
:104F7000F7B500231E285AD8384B8000C258042A9F
:104F80005BD007D8022A54D055D80423012A09D06F
:104F900000234CE0062A54D051D31A2A53D00223BE
:104FA0001B2AF5D12E4A116808294ED909294FD05C
:104FB0000A240226A02001252A4AC00015502A48AA
:104FC0002A4D07681C20BF00074029480197006848
:104FD0005759009027481B0207401F43C0230098E1
:104FE0009B020340FF2057515759000207401F43BF
:104FF000019B1F43009B58016023184007433E4319
:10500000565101251C4B156058680028FCD0002023
:105010005860A1230125DB00D3585560A025ED0081
:1050200050511BB2A14202D015D2611ACB401800D8
:10503000FEBD0823B6E71023B4E72023B2E74023E0
:10504000B0E78023AEE70123ACE708240026B1E7F0
:105050000C000126AEE7091B8B40E8E7B4A3000073
:105060002802002000700040E40100200405000038
:10507000E8010020FF00FFFFFC700040F0B51E2893
:105080005BD8364B8000C258354B1E68002E30D19D
:10509000C227344BBF00D859334C03250440C020ED
:1050A00000022043D851C0248020640080001851A1
:1050B0002E4F18602E4B803CD859FF3CA043D8514E
:1050C0000437D859A8432043D8510837D8590C354C
:1050D000A8438446072065462843D851A820C0002D
:1050E0001E50C1208026800076021E501C601C4B82
:1050F0001C60142500202B001E4C2E004643365900
:10510000771C1BD14343E250A0230325C132FF3259
:105110009200DB05D550184B1A68082A14D11423C5
:105120004343E3189A6812485132FF3292005960A3
:105130001150DA68C1239B00C250F0BD9642E1D005
:1051400001300328D9D1F8E7082A02D9083AD1401A
:10515000E5E708239A1A9140E1E7C046B4A30000AE
:105160004013002000E100E0FF00FFFF0405000005
:1051700000900040EC0100202C0200202149F0B5F5
:105180004A6C2148002A14D0A025A126002301241E
:10519000ED05F600C258571C06D0C7187F68002FCF
:1051A00002D027009740AF5114333C2BF2D100239B
:1051B0004B64A0230121DB0500260F009C4614232D
:1051C0004B43C3181A1F1268104C0E4D920014194D
:1051D0005219526C002A10D01A00143A1268551C49
:1051E00009D0103B1B68FF2B05D03B009340654660
:1051F0001A00074BEA50FC34666401310429DED101
:10520000F0BDC046FC900040EC0100200090004042
:105210000C05000000B51E2810D80C4A80008358E9
:1052200003290BD8A0220800C133FF33D2059B000D
:1052300001F000FA020905070021D15000BD0C2140
:10524000FBE70421F9E70321F7E7C046B4A3000018
:105250001E280AD8074B8000C25801239340A02281
:10526000D205002902D1044953507047A121C90039
:10527000FAE7C046B4A300000C05000003000020BC
:105280001E2B0AD8A021A222C905D2008858034AA1
:105290009B009B58D840012318407047B4A30000DE
:1052A0000849094A094B10B51B688858FA22190A9F
:1052B0001B0618439200002301F088FB4904C00B31
:1052C000084310BD001001400405000044130020F5
:1052D00070B5041E09D0FFF7E3FF050000F014F8D5
:1052E000FFF7DEFF401BA042F8D370BD0022044B45
:1052F0009A60044A13680133DBB213607047C046FA
:10530000FC100140441300207047000030B5214AD2
:105310004B0087B05B0893421EDD1F4A934205DDB8
:1053200002000B0002F08EFB07B030BD02AA00F0B5
:1053300035F803231840049A059B012813D002284E
:105340001DD0002814D00298039900F037FA80236A
:105350001B069C466144E7E70023002200930023DC
:1053600000F0A6FFE0E70298039900F027FADBE7D8
:10537000012402980399009400F09AFFD4E70124D5
:1053800002980399009400F093FF80231B069C462B
:105390006144C9E7FB21E93FFFFFEF7FF0B54E46CF
:1053A0004546DE465746E0B5E14B4C008FB090468F
:1053B000894664089C4200DC87E0DE4B9C4222DC8C
:1053C000DD4A002900DC92E0DC4B02F03BFBDB4BCA
:1053D00006000F009C4200D17EE1D94AD94B02F071
:1053E00031FB02000B00414630000A604B6039007F
:1053F00002F028FBD34BD24A02F024FB434601259E
:105400009860D9606BE0D04B9C4200DC8FE0CF4BC2
:105410009C4200DD55E1CE4A231592469A445146FE
:105420000905631A19001D00040002F053FE02F082
:1054300087FE02000B00200029000892099302F069
:1054400001FB0022C34B02F08BF80F00060002F0B4
:1054500041FE02F075FE04000D0002000B0030005A
:1054600039000A940B9502F0EDFA0022B94B02F0D4
:1054700077F8002200230C900D9101F079FA0028B2
:1054800000D192E1002300222000290001F070FAEF
:10549000434243410133B04A41460192022208A8E7
:1054A0000092524600F0A4FA4B460500002B16DA93
:1054B000802243461206944642465B684542634456
:1054C0005360D3686344D36009E00B000200414697
:1054D0000A604B600022002300258A60CB60280010
:1054E0000FB03CBC90469946A246AB46F0BD934BEC
:1054F00001F012FC914B06000F009C4200D13DE1EF
:105500008F4A904B01F008FC02000B00414630002E
:105510000A604B60390002F095FA894A894B01F024
:10552000FBFB012543466D429860D960D7E700F048
:1055300071FF8A4A8A4B06000F0002F011F8002220
:10554000884B01F0E9FB02F0C5FD050002F0F8FD13
:10555000794A7A4B0490059102F002F802000B00A0
:105560003000390002F06EFA754A06000F00049808
:105570000599744B01F0F4FF029003911F2D00DC9C
:10558000C7E0029A039B3000390002F05BFA8346C1
:105590008A4653465B0024155B0DE31A102B6CDD25
:1055A00004980599D322674B520501F0D9FF0200F8
:1055B0000B00300039000292039302F043FA0A0014
:1055C000010013000691079202003900300002F03A
:1055D00039FA029A039B02F035FA06000F0004988C
:1055E0000599614A614B01F0BBFF32003B0002F0BC
:1055F00029FA069E079F0B00020039003000029234
:10560000039302F01FFA4B005B0D83468A46E41AAF
:10561000312C32DD04980599B822544B920501F0E3
:105620009FFF03000C000200029303940B000698F6
:10563000079902F007FA02000B0006000F00069817
:10564000079902F0FFF9029A039B02F0FBF9484A1E
:105650000290039104980599464B01F081FF029A4C
:10566000039B02F0EFF902000B00300039000292B8
:10567000039302F0E7F983468A465A465346414669
:1056800030000A604B60390002F0DCF9029A039B9B
:1056900002F0D8F944460B000200A260E3604B46DA
:1056A000002B00DB1BE75B46236080231B06534473
:1056B000636080231B069C466144A060E1606D42EC
:1056C0000DE70B00020002F0BDF94346002598608B
:1056D000D9601860596002E7D3221A4B520502F0D4
:1056E000B1F9214A214B0D00040002F0ABF9020090
:1056F0000B00414620000A604B60290002F0A2F92D
:105700001A4B194A02F09EF9434601259860D96068
:10571000E5E602000B003000390002F093F96B1E41
:10572000154A9B009B5883468A46A342A5D130E781
:10573000FB21E93F7BD9024000004054FB21F93FA7
:105740003163621A61B4D03DFB213941FFFFEF7F25
:10575000EAFBFFFF00007041E0A4000083C8C96DB0
:10576000305FE43F0000E03F7370032E8A19A33BD3
:10577000C14920259A837B3960A40000D3220C4BB9
:10578000520501F0C9FA0B4A0B4B04000D0001F061
:10579000C3FA02000B00414620000A604B6029005A
:1057A00002F050F9034A044BB9E6032373E6C046FE
:1057B00061B4D03D7370032E8A19A33BF0B5474600
:1057C000CE4680B587B000920193754B4F0081465D
:1057D00088467F089F4263DC02F07CFC002800D1F1
:1057E000D4E04A4643464846414601F0B9FE04002B
:1057F0000D006C4A6C4B01F0B3FE6C4A6C4B01F02F
:105800008BFA22002B0001F0ABFE6A4A6A4B02F0D1
:1058100019F922002B0001F0A3FE684A684B01F041
:105820007BFA22002B0001F09BFE664A664B02F0D9
:1058300009F922002B0001F093FE644A644B01F049
:105840006BFA22002B0001F08BFE029003910022E4
:10585000604B2000290001F083FE029A039B0600A2
:105860000F002000290001F07BFE009A019B04003C
:105870000D004846414601F073FE02000B00200077
:10588000290002F0DFF802000B003000390002F0BE
:10589000D9F802000B0000204F4902F0D3F870E065
:1058A00002000B0001F05CFE04000D003D4A3E4B7F
:1058B00001F056FE3D4A3E4B01F02EFA22002B002D
:1058C00001F04EFE3B4A3C4B02F0BCF822002B009C
:1058D00001F046FE394A3A4B01F01EFA22002B0035
:1058E00001F03EFE374A384B02F0ACF822002B00A4
:1058F00001F036FE354A364B01F00EFA2B0022003D
:1059000001F02EFE354B029003919F429FDD344BF8
:1059100000229F423DDC334900207B182E491600AF
:105920001F0002F08FF8049005910022294B2000FF
:10593000290001F015FE32003B0002F083F8029AC4
:10594000039B06000F002000290001F009FE009AC9
:10595000019B04000D004846414601F001FE020093
:105960000B002000290002F06DF802000B0030004F
:10597000390002F067F802000B000498059902F064
:1059800061F807B00CBC90469946F0BD0020124962
:10599000F7E7154B002604920593144FC5E7C04660
:1059A000FFFF3F3ED43888BEE9FAA8BDC4B1B4BDFC
:1059B0009EEE213EAD529C804F7E923E9015CB19BB
:1059C000A001FA3E7751C1166CC1563F4C55555552
:1059D0005555A53F0000E03F0000F03F3233D33F74
:1059E0000000E93F0000E0FF0000E73F0000D23F79
:1059F000F0B5DE464E4645465746E0B5DC4CA5447C
:105A00000D9114001900A49A0993DA4B9200D6580C
:105A10004D1E03901821E01E0696029500F09EFE92
:105A2000C3430100DB1719404B1C9A009B1ADB0093
:105A30001B190B9105934C1B771918D4A59BA50036
:105A40009C463F1922AE6544013707E0286802F002
:105A500077FB013403C60435BC4208D0002CF5DACC
:105A600000200021013403C60435BC42F6D1069B58
:105A7000002B01DA00F0FDFB069B03990133DB00EC
:105A80009A46099BDA00944600920022914672AA37
:105A90000492B94A6144934688469AAB63449B4456
:105AA000029B002B00DABCE15D4600260027039C28
:105AB0004D442A686B6803CC01F052FD02000B00D4
:105AC0003000390001F028F9083D06000F00444578
:105AD000EFD1049B4B441E605F6008239C46E14469
:105AE000D145DDD10EA804218446494261448C464B
:105AF000069A93009C44614684460A910399083BA8
:105B000063448C460C93009B009263449B46009A2E
:105B10000498D10003008C46634408911E685F68B6
:105B2000002A33DD954980468C466244D300984470
:105B300070AB9A460EAB99460022914B300039006B
:105B400001F00EFD02F0C6FA02F0FAFA00228D4BC7
:105B500004000D0001F004FD02000B0030003900CC
:105B600001F070FF02F0B6FA4B4601C39946434676
:105B700020001A685B68290001F0CEF808235B4218
:105B80009C46E04406000F00D045D5D1059B30006F
:105B90001A003900984600F0DDFCFF2300229B0527
:105BA00004000D0001F0DCFC00F038FC0022764B14
:105BB00001F0D6FC02000B002000290001F042FF9A
:105BC0000D00040002F086FA814602F0B9FA0200E4
:105BD0000B002000290001F035FF060040460F00B1
:105BE000002800DCEEE0009B18215A1E92000EAB4C
:105BF0009B58091A1D000D41A9448D405D1B0EAB39
:105C00009D5017231B1A1D41002D2DDD01239C469D
:105C1000009BE144002B00DC1CE20E9C0123002CC5
:105C200000D0B5E0009A012A09D099000EAA545874
:105C30000133002C00D0ACE0009A9A42F5D1059BCC
:105C4000002B0EDD012B00D1A8E1022B09D1009B16
:105C50000EA95A1E92000EAB9B5807939B029B0AFB
:105C60008B50022D00D1C1E000230022300039000A
:105C700000F07EFE009B002800D194E2069A591E97
:105C80008A4210DC414A0A9894460EAA634494461C
:105C900000229B0063441C68043B22438342FAD1E8
:105CA000002A00D0C0E0069B0EAA013B9B00D358FF
:105CB000002B00D0B3E001220C9B043B5968013259
:105CC0000029FAD0009B9C466244110007921A00FA
:105CD00001338B4246DC0B9863468046A59C4344C7
:105CE000A046099C9B00A1464A449844D30022AA9E
:105CF0009146049A99449446089BA59A6344844625
:105D0000614494469A468B00634400934346586826
:105D100002F016FA4B4618605960029B002B24DBF8
:105D20004D46039C0026002701E0286869680CCCDA
:105D300001F016FC02000B003000390000F0ECFF0F
:105D4000083D06000F005C45EFD153469E60DF60C2
:105D500004239C460433E0449C46009BE144E24417
:105D60009845D3D1079B0093D1E600260027ECE7A6
:105D700094FDFFFF28A6000018FEFFFFFFFFFF1F96
:105D80000000703E0000704100002040FFFFFF3F18
:105D9000002180225204141B0EAA545000999942EB
:105DA0000EDD0EA884469B000EAA8900D2586144DD
:105DB0006344CF4800E01A68821A04C38B42FAD1C8
:105DC00001243CE7059B002B06D1009B0EAA013B5A
:105DD0009B00D558ED1517E70022C64B300000F0A8
:105DE000EBFD002800D024E100253DE732003B0018
:105DF0000020C14901F026FE06000F00002C00D152
:105E000032E7059A0020BC4900F0A4FB02000B0019
:105E10003000390001F016FE06000F0024E70122D1
:105E200050E70026002754E64B46059A079388461C
:105E30008B000EA9CB58183A08950592002B0DD16E
:105E40008C464146AD4B43449B006344043B586839
:105E50000139183A0028F9D088460592059A0020A1
:105E6000A54900F077FB434604000D00002B00DA43
:105E700005E29E000EAB9C464346DB0066449C4612
:105E8000059370AB9946049F67440097306802F011
:105E900057F922002B0001F063FB00223860796083
:105EA000974B2000290001F05BFB083F04000D0028
:105EB000043EB945EAD14AAB03939B4600239A4678
:105EC000069B4246994643460132029204934B4652
:105ED000002B00DAAAE080208A4B009D9846C0057E
:105EE000894900260027002408E008239C4608353D
:105EF000E044544511DC4346186859682A686B68C9
:105F000001F02EFB02000B003000390000F004FF0E
:105F1000013406000F00A145E7DA5B46C0C39B468B
:105F200001239C46009BE244083B0093029B9A4558
:105F3000CDD1049B9846A49B022B00DD8EE0002B64
:105F400037DC1FD1059B00271D00039B00249C46C6
:105F50001E006544083E2A686B683800210000F086
:105F6000DBFE083D07000C00AE42F4D1089B002B7D
:105F700003D080231B069C4664443A0023000D99FD
:105F80000A604B600720079B18409B239B009D44A1
:105F90003CBC90469946A246AB46F0BD009B0EA97C
:105FA0005A1E92000EAB9B5807935B025B0A8B5004
:105FB00057E64346002B00DA70E100200021DB00A9
:105FC0004AAAD61848AF32687368083E00F0A4FEAB
:105FD000B742F8D1089B002B00D025E10B0002004E
:105FE0004A984B990D9C2260636001F02BFD43465B
:105FF00007000C00002B13DD01254CAEB146380024
:106000002E0021004C4601360CCC00F085FEA14646
:10601000B045F7DA089B07000C00002B00D015E113
:106020003A0023000D998A60CB60ABE70026002779
:1060300073E701239C46009BE1440225002B00DD11
:10604000EBE532003B0000202B4901F0FBFC060091
:106050000F0009E60024F2E54AAB0393A49B032B4F
:1060600000D08FE74346002B00DC14E1039ADB00ED
:106070009B46130091465B441E685F68234B434474
:106080000293DB00994448AB9A464B465C681B6818
:106090001800210032003B000090019100F03CFE0E
:1060A00004000D0002000B000098019901F0CAFCE9
:1060B0003B00320000F030FE4B469860D9601C6017
:1060C0005D6008235B429C46E14426002F00CA45E0
:1060D000DBD14346012B00DCE3E0039A13005B4471
:1060E0001E685F68029BDB0099464A44904610E0B8
:1060F000FFFFFF000000E03F0000F03FFFFFFF3F19
:106100000000703EE8A50000FB21F93FFFFFFF1FE4
:10611000984643465C681B681800210032003B002B
:106120000090019100F0F8FD04000D0002000B004A
:106130000098019901F086FC32003B0000F0ECFD74
:106140004346039A9860D9601C605D60083B260056
:106150002F009A42DCD14D46944600260024474643
:10616000083565442A686B683000210000F0D4FDD2
:10617000083D06000C00AF42F4D1039B4A9F5D68C6
:106180009968D868089B002B65D080221206944637
:106190000D9B6544604464441F605D609960D860F5
:1061A0001E615C61EEE69A464B460793059B300004
:1061B0005A423900089500F0CDF900223A4B06000A
:1061C0000F0000F0F9FB002824D0384B00223000EB
:1061D000390001F0C5F901F07DFF52460400950039
:1061E00001F0AEFF0022304B01F0BAF902000B00C3
:1061F0003000390001F026FC01F06CFF0EAA50516E
:106200000122059B524418339046059393000EAA31
:10621000D45023E65346300039009C0001F05AFF69
:106220000EAB1851D04619E680230D9A1B06CB18E9
:10623000106053600B0002004A984B9901F002FC79
:10624000434607000C00002B00DDD5E680231B062B
:106250009C466444E4E62B003A000D9D2A606B6086
:106260000A000300AA60EB60320023002A616B6120
:1062700088E6099BDB00009372AB049332E4A49B95
:10628000022B00DDE8E6002B00DD92E600D079E687
:10629000002700246AE6002600246EE70020002183
:1062A00098E60026340068E7000070410000703E68
:1062B000F0B5CE46474680B587B000920193474A75
:1062C0004B00814688465B08934207DC41464846BE
:1062D00001F000FF4146031E484666D04A46434649
:1062E0004846414601F03CF904000D0002000B0055
:1062F0004846414601F034F9394A3A4B06000F004E
:106300002000290001F02CF9374A384B01F09AFBA4
:1063100022002B0001F024F9354A364B00F0FCFC3A
:1063200022002B0001F01CF9334A344B01F08AFBA8
:1063300022002B0001F014F9314B324A00F0ECFC42
:106340000E9B02900391002B34D0009801990022FB
:106350002D4B01F005F9029A039B04900591300042
:10636000390001F0FDF802000B000498059901F0D6
:1063700069FB22002B0001F0F3F8009A019B01F069
:1063800061FB224A04000D00214B3000390001F06E
:10639000E7F802000B002000290000F0BDFC02001D
:1063A0000B004846414601F04DFB07B00CBC90463F
:1063B0009946F0BD02000B002000290001F0D0F842
:1063C000124A134B01F03EFB32003B0001F0C8F8CB
:1063D0004A46434600F0A0FCE7E7C046FFFF3F3EC9
:1063E0007CD5CF5A3AD9E53DEB9C2B8AE6E55A3E5F
:1063F0007DFEB157E31DC73ED561C119A0012A3FFB
:106400001111813FA6F810110000E03F4955555584
:106410005555C53F49004B0819007047474AF0B52C
:106420004F4691464B005B0D99444646D6464A4638
:10643000C0B505000C000E0088460700132A27DCB3
:10644000002A4BDB3E4B13419A460B005246134049
:10645000034318D03B4A3C4B2800210000F05CFC71
:106460000022002300F09EFA002847D0002C04DA16
:1064700080234A465B03134198444646534600270F
:106480009E43380031001CBC90469946A246F0BDA0
:10649000332A08DD8023DB009945F4D102000B008C
:1064A00000F03AFCEFE7294A944601226344524245
:1064B000DA4092460242E6D0224A234B28002100CD
:1064C00000F02AFC0022002300F06CFA002815D00E
:1064D000002C1EDB534646469F430FE0194A1A4BD9
:1064E0002800210000F018FC0022002300F05AFAD6
:1064F000002803D0002C04DB0027002638003100E0
:10650000C1E76400640825430027002DF6D0104E33
:10651000F4E74B46142B0BD03422D21A01239340BC
:106520005D19BD4208D201239C462F00E044D1E70B
:10653000133B9C46E044CDE72F00CBE701FCFFFF77
:10654000FFFF0F009C7500883CE4377EEDFBFFFFEA
:106550000000F0BF4B0070B55B0D14000A00002B6B
:106560001AD14B005B08034315D0234B002200F0E7
:10657000F7FF224B9C422DDB0A004B005B0D363BA4
:106580001F4DE318AB422ADC002B0DDD1D4C1B0513
:1065900022401A43110070BD1B4DAB42F0D10200E6
:1065A0000B0000F0B9FBF6E71D00353519DA174B83
:1065B00002009C4209DD0B001548164900F032F834
:1065C000134A144B00F0CCFFE5E70B0012481349C7
:1065D00000F028F8104A114B00F0C2FFDBE7020080
:1065E000E9E7084C363322401B051343190000220B
:1065F0000B4B00F0B5FFCEE700005043B03CFFFF6F
:10660000FE070000FFFF0F80FF07000050C30000DF
:106610009C7500883CE4377E59F3F8C21F6EA501D3
:106620000000903C30B54A00DB0FDB0752081A43EC
:10663000110030BD02B4714649084900095C4900A7
:106640008E4402BC7047C046002243088B4274D37C
:1066500003098B425FD3030A8B4244D3030B8B4263
:1066600028D3030C8B420DD3FF22090212BA030C6C
:106670008B4202D31212090265D0030B8B4219D34D
:1066800000E0090AC30B8B4201D3CB03C01A52416D
:10669000830B8B4201D38B03C01A5241430B8B42B5
:1066A00001D34B03C01A5241030B8B4201D30B039E
:1066B000C01A5241C30A8B4201D3CB02C01A5241C5
:1066C000830A8B4201D38B02C01A5241430A8B4288
:1066D00001D34B02C01A5241030A8B4201D30B0271
:1066E000C01A5241CDD2C3098B4201D3CB01C01A8B
:1066F000524183098B4201D38B01C01A5241430995
:106700008B4201D34B01C01A524103098B4201D382
:106710000B01C01A5241C3088B4201D3CB00C01AEF
:10672000524183088B4201D38B00C01A5241430867
:106730008B4201D34B00C01A5241411A00D201468C
:10674000524110467047FFE701B5002000F0F0F815
:1067500002BDC0460029F7D076E7704703460B43D9
:106760007FD4002243088B4274D303098B425FD34A
:10677000030A8B4244D3030B8B4228D3030C8B4276
:106780000DD3FF22090212BA030C8B4202D312125C
:10679000090265D0030B8B4219D300E0090AC30B31
:1067A0008B4201D3CB03C01A5241830B8B4201D3DE
:1067B0008B03C01A5241430B8B4201D34B03C01AC7
:1067C0005241030B8B4201D30B03C01A5241C30A3F
:1067D0008B4201D3CB02C01A5241830A8B4201D3B0
:1067E0008B02C01A5241430A8B4201D34B02C01A9A
:1067F0005241030A8B4201D30B02C01A5241CDD23F
:10680000C3098B4201D3CB01C01A524183098B4289
:1068100001D38B01C01A524143098B4201D34B0172
:10682000C01A524103098B4201D30B01C01A5241D5
:10683000C3088B4201D3CB00C01A524183088B425C
:1068400001D38B00C01A524143088B4201D34B0045
:10685000C01A5241411A00D20146524110467047B7
:106860005DE0CA0F00D04942031000D340425340BC
:1068700000229C4603098B422DD3030A8B4212D37C
:10688000FC22890112BA030A8B420CD389019211AE
:106890008B4208D3890192118B4204D389013AD0EB
:1068A000921100E08909C3098B4201D3CB01C01AC0
:1068B000524183098B4201D38B01C01A52414309D3
:1068C0008B4201D34B01C01A524103098B4201D3C1
:1068D0000B01C01A5241C3088B4201D3CB00C01A2E
:1068E000524183088B4201D38B00C01A5241D9D246
:1068F00043088B4201D34B00C01A5241411A00D2C7
:106900000146634652415B10104601D34042002BC2
:1069100000D54942704763465B1000D3404201B541
:10692000002000F005F802BD0029F8D016E77047F6
:106930007047C046D0400B1C1141203A03D49C46FE
:106940001341184363465242934018437047C04670
:106950008446101C62468C46191C634600E0C04603
:106960001FB500F095FD002801D40021C8421FBDCD
:1069700010B500F0EDFC4042013010BD10B500F044
:1069800087FD002801DB002010BD012010BDC0469E
:1069900010B500F07DFD002801DD002010BD0120B4
:1069A00010BDC04610B500F00FFD002801DC00202E
:1069B00010BD012010BDC04610B500F005FD002837
:1069C00001DA002010BD012010BDC046F0B5CE4652
:1069D000474615042D0C2E0080B50704140C3F0CFF
:1069E0009946030C7E435D43674363437F19340C30
:1069F000E4199C46A54203D980235B029846C4440F
:106A00004B4643435143250C36046544360C24045D
:106A1000A4195B19591820000CBC90469946F0BD8A
:106A2000F0B54E4657464546DE46E0B543025B0AA2
:106A3000450083B00F1C99462D0EC60F002D57D070
:106A4000FF2D24D08020DB00C004184300238146A2
:106A50009A469B467F3D7C027A00FB0F640A120E29
:106A6000984623D0FF2A4BD0E30080240020E40482
:106A70007F3A1C43AD186B1C474601935346774041
:106A80003A000F2B48D87D499B00CB589F46002BDE
:106A900000D085E008339A46063B9B467C027A008C
:106AA000FB0FFF25640A120E9846DBD1002C00D0A4
:106AB00090E0524601231A4392460120DBE74C4600
:106AC00058461700022824D0032800D1CFE0002226
:106AD000002301284DD15802D205400AFF07104378
:106AE000384303B03CBC90469946A246AB46F0BD45
:106AF000002B5BD104239A46033B00259B46AAE763
:106B0000FF35002C60D1524602231A4392460220E0
:106B1000B1E7FF220023DEE74B461B0C9C464B46A9
:106B20002604360C180461463300220C6446000C1F
:106B300043434E435043544380191A0C1218964253
:106B400003D9802149028C4664441B041B0C1004A9
:106B5000C01883015E1EB341800E1843130C1B192D
:106B60009B0103431C00230179D5012362081C40CB
:106B70001443019A7F32002A4DDD630704D00F23AE
:106B80002340042B00D00434230103D53C4B019A4D
:106B90001C408032FE2ABCDCA3015B0AD2B29AE719
:106BA0000C239A46093BFF259B4654E7180001F049
:106BB00053FB4A46431F76259A4000236D42914677
:106BC0002D1A9A469B4646E7524603231A4392469D
:106BD000032050E7200001F03FFB431F2D1A9C408B
:106BE000763D002047E780230027DB03FF2272E782
:106BF000424666E74C463200584662E780234A46E2
:106C0000DB031A4222D01C4220D123435B025B0AE1
:106C10004746FF225FE701239A1A1B2A21DC230043
:106C20000199D3409E318C401A0023005C1EA34181
:106C300013435A0704D00F221A40042A00D0043309
:106C40005A0111D49B015B0A002244E780234A4683
:106C5000DB0313435B025B0A3700FF223BE701952E
:106C600087E70022002336E70122002333E7802351
:106C7000DB0323435B025B0AFF222CE738A60000FC
:106C8000FFFFFFF770B500283DD0C317C5185D4062
:106C9000C40F280001F0E0FA9E22121A962A07DC9F
:106CA000D2B2082833DD083885406802400A23E064
:106CB000992A0BDD052329001B1AD94003001B3339
:106CC0009D402B005D1EAB4119430D00052801DDE1
:106CD000431F9D402B000F490B406E0709D00F2624
:106CE0003540042D05D004335D0102D59F220B40B1
:106CF000121A9B01580AD2B24002D205400AE40798
:106D00001043204370BD002400220020F4E76802F5
:106D1000400AF1E7FFFFFFFBF0B54F464646D64677
:106D20000C000903C0B5490A470F5E0039431F0331
:106D3000DB0F9C4665007B0A570F1F436D0DE40F68
:106D4000760DA146C000B846D200AB1B64457BD08F
:106D5000002B5FDD002E00D0A4E03E00164300D1E2
:106D600012E15E1E002E00D09EE1871A4346B84213
:106D700080410125C91A4042091A0B0200D431E1B1
:106D800049024E0A002E00D16EE1300001F064FA93
:106D90000300083B1F2B00DD61E120223900D21ADD
:106DA0009E40D1409F400E439D4200DD51E15D1B5E
:106DB0006B1C1F2B00DD7CE12021C91A3D00300037
:106DC0008F408840DD40791E8F41310007222843E3
:106DD000D940002507433A40002A09D00F233B4001
:106DE000042B05D03B1DBB42BF417F42C9191F0088
:106DF0000B0200D426E26A1CC64B55056D0D9A4263
:106E000000D106E1C44AFF080A40530752023B433F
:106E1000120B8EE0002B00D0B8E06B1C5B055B0D05
:106E2000012B00DC30E1871A4346B842B641CB1A49
:106E300076429E1B330200D54CE13B003343A1D187
:106E400000220024002570E0002B00DCE5E0002E8D
:106E500000D183E0AF4EB54260D080263604374380
:106E6000B846382B00DC3EE1434613431F007A1E30
:106E700097413F1887428041404209180B0200D4D5
:106E8000B0E0A44B01359D4200D1C3E0A24A7B088B
:106E90000A4001210F401F435108D30707221F4317
:106EA0003A4099E79B4EB54238D0802636043743A6
:106EB000B846382B00DDDCE01F2B00DC30E11E0083
:106EC0004746203EF740BC46202B04D04026F31A0C
:106ED00046469E403243170063467A1E97411F4341
:106EE000CCE0002B00D104E24346134300D159E12A
:106EF0004B07C00818438023C9081B03194208D058
:106F00004546ED081D4204D14346D00859070843C1
:106F10002900420FC9007F4D1143C0004B07CA082A
:106F20007C49C00803438D4268D012036D05120BE3
:106F30006D0D002112031800130B0A0D12051A43E0
:106F4000764B2D0513402B435B00E4075B0823437E
:106F500019001CBC90469946A246F0BD3E0016435F
:106F600012D05E1E002E00D000E1871887428041BB
:106F700041444042091801250B0233D5022585E71B
:106F800064463300414610001D00C7E7002D00D0C5
:106F9000DAE00C000443F3D05C1C00D19FE15D4CAF
:106FA000A64200D12FE1DB43382B00DD66E11F2B29
:106FB00000DD83E120240500E41A0F00DD40D94004
:106FC000A0404346A7405B1A441EA04198462F4369
:106FD0003843171ABA42924143465242991A6446BC
:106FE0003500CAE607223A40002A00D0F6E64B07F1
:106FF000CA084849FF083B438D4296D11900114306
:1070000000D19EE1802109030A431203120B414D76
:107010008FE71500002200238BE7002B00D0C7E08C
:107020006B1C5F057F0D012F00DCF1E0394DAB4299
:1070300000D1B9E085180A0085428941424449429D
:1070400051180722CF076D082F4349083A401D0009
:10705000C2E607223049ED1A31403A40BCE63E0014
:107060002838864000279FE6380001F0F5F82030E8
:107070008EE6434613431F007A1E9741C71BB84252
:1070800080414042091A78E60E003B000643134354
:10709000002D61D1002E00D0F4E0002B00D11BE1C7
:1070A00064463900100039E71A4FBB427AD03300EA
:1070B000FFE630001F3DE840202B03D04021CB1AD3
:1070C0009E4037437B1E9F41072207433A400021E1
:1070D000002589E7171A4346BA42B641591A764243
:1070E0008E1B64464EE61F2B00DDADE02026474692
:1070F000F61AB740B9461700B246DF404E463E4347
:1071000037005646B240561EB24117434246DA4057
:107110008918AEE6FF070000FFFF7FFFFFFF0F802B
:1071200020264746F61AB740B9461700B246DF4058
:107130004E463E4337005646B240561EB2411743B4
:107140004246DA40891A99E77F4CA6425BD08024F8
:1071500024045B42214327E7002E0CD1002B00D1F1
:10716000CBE0644639001000774DD7E6764FBB423E
:1071700018D0330075E6002B14D04B07C008184315
:107180008023C9081B03194207D0FC081C4204D104
:107190007907D0080843E14621004C46420FC90058
:1071A0001143C000684DB9E61D0000220023C0E66F
:1071B000002D5BD10D00054300D1E2E65D1C00D13E
:1071C000B0E0614DAE421FD0DB43382B71DC1F2B8A
:1071D00000DD96E020250F00ED1AAF40B94607000C
:1071E000AA46DF404D463D432F005546A840D940B2
:1071F000451EA84188440743BF1897429241514217
:10720000414435003AE6644635004146100085E6C3
:107210000B000343002D00D063E6002BF5D043465E
:10722000134300D17AE68718874280410722414400
:10723000404209183A400B0200D4D5E6434B0135D1
:107240001940C9E5380069E61E004746203EF74070
:10725000BC46202B04D04026F31A46469E403243BB
:10726000170063467A1E97411F4302E6364DAE4231
:10727000CAD080252D045B422943A6E70843411E5E
:107280008841A6E6002B00D148E6871A4346B8425B
:10729000B641CB1A76429E1B33024BD5171A434692
:1072A000BA429241591A5242891A072264463A4018
:1072B00092E501430F00791E8F419DE71C000F00EE
:1072C000203CE740202B03D04024E31A9940084398
:1072D000411E884138437CE60022002425E6171A27
:1072E0004346BA429241591A5242891A64463500BD
:1072F00043E541461000144D10E68022002412039D
:1073000080E61D000F00203DEF40BC46202B03D03F
:107310004025EB1A9940084307006346781E8741D1
:107320001F4369E7871897429B4141445B42C91854
:107330003500A3E53B003343CED0072231003A406D
:1073400052E600231A00F4E5FF070000FFFF7FFF6D
:10735000F0B54F464646D6468446C0B58046194EDF
:1073600018030F034D00000B5C0082463F0B6D0DB0
:10737000C90F9146640DDB0F0120B5420AD0B4421B
:1073800003D0A54201D157450CD01CBC904699466C
:10739000A246F0BD66463E43F7D1AC42F5D1544615
:1073A0001443F2D10120C845EFD1994207D0002DF6
:1073B000EBD163461F433800471EB841E5E7002084
:1073C000E3E7C046FF070000F0B54F464646D64605
:1073D0004D00C0B50E03C90F8A462C491F035C003F
:1073E0008046360B6D0D91463F0B640DDB0F8D42D1
:1073F0001ED08C4216D0002D1ED130438446002C66
:1074000001D13A4323D06246002A1AD09A4529D0A6
:10741000514602200139084001381CBC904699466B
:10742000A246F0BD39001143E5D002204042F4E706
:107430003043FAD1AC420FD0002C0FD13A43E7D001
:107440000CE00122013B934318000130E5E763465D
:107450000020002BE1D0DBE73A43E6D19A45D7D1B3
:10746000A542D5DCA54205DBBE42D1D808D000201C
:10747000BE42D2D250460123013898430130CCE7B6
:10748000C845C5D80020C845F4D3C6E7FF070000AB
:10749000F0B54F464646D6464D00C0B50E03C90F5F
:1074A0008A462E491F035C008046360B6D0D9146BF
:1074B0003F0B640DDB0F8D4218D08C4211D0002D94
:1074C00018D130438446002C1ED13A431CD1634668
:1074D0000020002B30D051460220013908400138ED
:1074E0002AE039001143EAD0022025E03043FBD1E5
:1074F000AC4226D0002C26D13A4324D1514602205A
:1075000001390840013817E06246002A0FD09A4539
:10751000E1D1A54205DBBE42DDD819D00020BE4234
:107520000AD25046012301389843013004E0012279
:10753000013B9343180001301CBC90469946A2467B
:10754000F0BD3A43D0D19A45C5D1A542C3DCE0E7AE
:10755000C845C0D80020C845E3D3EDE7FF070000C9
:10756000F0B55746DE464E464546E0B58346060032
:107570000F03480087B092461D003F0B400DCC0F13
:10758000002800D16FE0DE4B984238D08023FF0006
:107590001B041F43730F3B430193DA4B00279946AB
:1075A00000239B46F60081442B0369001B0B5246C7
:1075B0009846490DED0F002900D185E0D04B994246
:1075C00000D173E04346DA0080231B041343524684
:1075D000CC48520F84461343524600206144D200E7
:1075E00089442100694000918C46012149448A4622
:1075F0000F2F00D990E0C449BF00CF59BF465B466A
:107600003B43019300D06AE102230827002681460C
:107610009B46C9E732005846019B6146009102280B
:1076200000D175E0032800D1FEE1012800D02CE153
:1076300000230027002600253F032A0D3F0BB348F7
:1076400012053A4302401B051343009A5B00D10721
:107650005B080B433000190007B03CBC90469946CC
:10766000A246AB46F0BD5B463B43019300D12FE100
:10767000002F00D1A5E1380000F0EEFD03000B3B28
:107680001C2B00DD96E11D22D31A5A460100DA4078
:107690005E4608398F4013008E403B4301939C4B5C
:1076A00000271B1A994600239B467DE74146534617
:1076B0000B4393498C46E144002B00D01AE102228F
:1076C0000220174300228CE7134300D10DE143460B
:1076D000002B00D181E1404600F0BEFD02000B3AD4
:1076E0001C2A00DD72E10100434608398B409846B0
:1076F0001D239A1A5346D3401A0043461343524659
:107700008A404946081A824989468144002068E730
:107710007B4B002700268EE7140C1204120C11007C
:10772000370C3604350C794328008C462E00604314
:107730006044834656432100300C804658467943C6
:1077400040440291844506D98846802149028C46EE
:10775000E044414602913604010C360C00048B468D
:1077600081191E0C1B041B0C0391190079438C46D4
:10777000280075436544A8465843050C45447743A3
:10778000A94203D9802149028C466744290C8C46C2
:1077900039000004000C2D042D186144AB44059100
:1077A0005946049101990F043F0C080C39005143CC
:1077B0004243904602008C46090C8B4662437C4350
:1077C00044445C44A04503D9802149028846424490
:1077D000210C884661460904090C8C46390059433E
:1077E000434370437E430F0CF6182404BE196444CF
:1077F00042448C46B34203D980235B0298464044FE
:10780000029B61469846049B370443449B46AB4524
:10781000AD416B420D0405992D0C8C467F196744D0
:10782000FD18A8465D462D19A542A4419346644221
:10783000A446C344DC448F42BF4198459B419345D5
:107840009241A445A4415B427F421F43360C524201
:107850006442BF192243BF18624638184302D20D52
:10786000039913436A020A43501E82416146ED0D9B
:107870002A434E023243D90100D4B3E00126500816
:1078800032400243DE0732435B08224C5444002C52
:1078900062DD510709D00F201040042805D0101DCB
:1078A0009042924152429B180200D90104D5802493
:1078B0001948E400034054441848844200DD27E797
:1078C0005E075B02D2081F0B630516435B0DB2E631
:1078D000002399460133042700269B4664E60323D0
:1078E000019781460C279B465EE601220120174343
:1078F000002276E6032303201F43434671E6C04679
:10790000FF07000001FCFFFF78A60000FFFF0F80CB
:107910000DFCFFFFFF030000FFFFFFFEFE0700005E
:107920000023802700933F030026434B83E6019BFF
:107930003200A446584670E6AC466EE680270199B0
:107940003F0339422DD03B422BD11F433F033F0B16
:1079500000951600384B6EE601252D1B382D00DDF5
:1079600066E61F2D40DC35481C005044160082405E
:107970008440EE40501E824134431443EB40620782
:1079800009D00F222240042A05D02200141D94425F
:10799000804140421B181A023ED5012300270026D1
:1079A00049E68027019B3F031F433F033F0B0094A1
:1079B000214B40E603005A46283B9A40002601929C
:1079C0006DE6584600F048FC203057E6030052466A
:1079D000283B9A401300002293E6504600F03CFCFE
:1079E00020307BE6CA4650E71F201E004042041BA1
:1079F000E640202D03D0124C5444A3401A43501E9D
:107A00008241324307260027164009D00F20002369
:107A1000104014000428B9D122005E075B021F0B3E
:107A2000D2081643002306E680273F031F433F0387
:107A30003F0B1600004BFEE5FF0700001E04000090
:107A40003E040000F8B557464E464546DE460C005B
:107A50000903E0B5490A460F5F0031431E03DB0FFF
:107A6000760A9B46530F3343C84E6500C000E40FAF
:107A7000D2006D0DA24681467F0D9C469046B742CE
:107A800000D1B9E05B46012673409B46EE1BA3453F
:107A900000D183E0002E63DD002F00D0B1E063460B
:107AA000134300D123E1731E002B00D0BAE1861AE4
:107AB0006346B04280410125C91A4042091A0B02AF
:107AC00000D447E149024B0A98464346002B00D1B7
:107AD00089E1404600F0C0FB0300083B1F2B00DD9E
:107AE0007CE120223000D21A4146D0409940020069
:107AF0009E400A439D4200DD6AE15D1B6B1C1F2B0B
:107B000000DD94E1202110003500C91A8E40DA40D2
:107B10008840DD40711E8E41110007222843002558
:107B200006433240002A09D00F233340042B05D0EE
:107B3000331DB342B641764289191E000B0200D4B0
:107B40003DE26A1C914B55056D0D9A4200D119E139
:107B50008F4AF6080A40570752023743120B9BE040
:107B6000002E00D0C5E06E1C7605760D012E00DCDF
:107B700048E16746861ACB1BB042BF417F42B846F8
:107B80001F004346FF1A3B00B8461B0200D55FE1C9
:107B900037439AD100220024002579E0002E00DC32
:107BA000FAE0002F00D18DE0784B9D4267D0802312
:107BB00067461B041F43BC46382E00DC52E1634677
:107BC00013435A1E93411E188642804140420918B1
:107BD0000B0200D4BEE06D4B01359D4200D1D2E0D6
:107BE0006B4A73080A4001210E401E435108D30717
:107BF00007221E43324095E71E00164300D045E79A
:107C000040E7624B9D423AD0802367461B041F43E6
:107C1000BC46382E00DDEBE01F2E00DC3AE13300DD
:107C20006746203BDF403B00202E05D04027BF1B8E
:107C30006646BE40324390464646721E96413343E6
:107C4000DAE0002B00D114E26346134300D168E16F
:107C500080234E07C008C9081B030643194208D0F9
:107C60006046C008184204D163460100D2085E078E
:107C70001643F3009946C900720F444D11434B4619
:107C8000DE08424B4F073743CA089D4200D16EE0E1
:107C900012036D05120B6D0D00211203130B0A0D5B
:107CA00012051A433B4B2D0513402B435B00E407A1
:107CB0005B082343380019003CBC90469946A24615
:107CC000AB46F8BD6346134311D0731E002B00D0A2
:107CD00007E1861886428041614440420918012527
:107CE0000B0237D502257BE73E0061469146350001
:107CF000C5E75C46002D00D0E1E00B000343F3D064
:107D0000731C00D1ACE1214B9F4200D13AE1F34317
:107D1000382B00DD6FE11F2B00DD8CE120250E00EC
:107D2000ED1AAE40B0460600AA46DE404546354351
:107D30002E005546D940A8406346451EA8415B1A0F
:107D40009C463043161AB242924163465242991AF7
:107D50003D00B4E607223240002A00D0E4E60B4B97
:107D6000F6084F073743CA089D4200D090E73B0012
:107D7000134300D1A6E180231B031A431203120B05
:107D8000024D89E715000022002785E7FF07000064
:107D9000FFFF7FFFFFFF0F80002E00D0C7E06B1CAE
:107DA0005E05760D012E00DCF0E0C84DAB4200D13F
:107DB000B9E085180A008542894162444942511858
:107DC0000722CE076D082E43490832401D00A9E660
:107DD000BF49ED1A114007223240A3E6320028388D
:107DE0008240002686E6300000F036FA203073E646
:107DF000634613435A1E9341C61AB0428041404223
:107E0000091A5CE60E00674606431743002D5ED153
:107E1000002E00D0F3E0002F00D11EE15C46614649
:107E200091462CE7A94FBE427BD01E00F1E6100020
:107E30001F3DE840202B03D04021CB1A9A40164327
:107E4000731E9E410722064332400021002583E72E
:107E5000161A6346B2428041591A40420B1A98469C
:107E60005C4632E61F2E00DDABE02027BB1B9A46A6
:107E700063465746BB40994613004F46F3401F43A5
:107E80003B005746BA40571EBA4113436246F24080
:107E9000891898E62027BB1B9A4663465746BB4085
:107EA000994613004F46F3401F433B005746BA40E4
:107EB000571EBA4113436246F240891A9CE7834B2E
:107EC0009F425FD080252D047342294320E7002E76
:107ED0000CD1002F00D1D0E05C46614691467B4D2D
:107EE000CDE67A4FBE421CD01E0065E6002F18D0AA
:107EF000C0084E0706438020C9080003014208D08D
:107F00006346DC08044204D12100DA46D2085E0749
:107F10001643F300994601245346C900720F1143DA
:107F20001C406A4DABE61D0000220027B4E6002D80
:107F300059D10B00034300D1D6E6731C00D1B2E047
:107F4000624B9F421ED0F343382B6FDC1F2B00DDAA
:107F500097E020250E00ED1AAE40B0460600AA4676
:107F6000DE40454635432E005546A840D940451EC3
:107F7000A8418C440643B61896429241514261444E
:107F80003D0025E63D006146914678E60B0003433F
:107F9000002D00D055E6002BF5D06346134300D1E9
:107FA0006DE68618864280416144404209180022ED
:107FB0000B0200D4D0E6464B01351940B2E5B1467C
:107FC0005DE633006746203BDF403B00202E05D0B6
:107FD0004027BF1B6646BE40324390464646721E4F
:107FE00096413343EFE5394B9F42CBD080252D049A
:107FF00073422943A8E70843411E8841A2E6002FA7
:1080000000D13CE66346861ACF1AB0429B415B42E0
:10801000FB1A98461B024ED5161A6346B24292418D
:10802000591A5242891A5C4600227BE501430E0030
:10803000711E8E419FE71D000E00203DEE40B046B0
:10804000202B04D04025EB1A99400843814648462E
:108050004346411E8841184374E60022002417E677
:10806000161A6346B2429241591A5242891A3D0089
:1080700025E561469146154D01E680220024120354
:1080800079E61D000E00203DEE40B046202B04D0C6
:108090004025EB1A9940084381464E464346711EDF
:1080A0008E411E4367E7861896429B4161445B42BE
:1080B000C9183D008CE547463743CED007224146DC
:1080C000324049E600273A00E6E5C046FF070000D7
:1080D000FFFF7FFF30B5144D0A034B00120B5B0D01
:1080E000C90F0024AB4211DD104CA34210DC8024E8
:1080F000640322430E4CE41A1F2C0CDD0D48C31AF6
:10810000DA4013005C42002900D11C00200030BD81
:10811000094BCC18FAE7094DE040AC4663449A405D
:1081200013000343EEE7C046FE0300001D040000F9
:108130003304000013040000FFFFFF7FEDFBFFFF8F
:1081400070B500282DD0C317C5185D40C40F280096
:1081500000F082F8154B1B1A5B055B0D0A2815DD34
:108160000B38854000222D032D0B002110002D031C
:108170000A0D2D0B12052A430D4D1B052A401343F2
:108180005B00E4075B082343190070BD020029006F
:10819000153291400A000B21081AC5402D032D0B02
:1081A000E3E70024002300250022DEE71E04000090
:1081B000FFFF0F804100090E4B1C70B5DBB2460279
:1081C000750AC40F012B14DDE0239B006D07360BED
:1081D000CB1800210A0D280012051C4D32435B0507
:1081E0002A405B0813435B00E4075B082343190044
:1081F00070BD002914D1002D1ED0280000F02CF8ED
:108200000A281CDC0B232A001B1ADA400300153352
:108210009D400F4B12031B1A5B05160B5B0DD8E735
:10822000002D06D0320B802636036D071643094B0E
:10823000CFE7084B0026CCE700230026C9E7030060
:108240002A000B3B9A400025E3E7C046FFFF0F8062
:1082500089030000FF0700001C2101231B04984232
:1082600001D3000C10391B0A984201D3000A0839C7
:108270001B09984201D30009043902A2105C40187E
:108280007047C04604030202010101010000000022
:108290000000000030B51C00094B05001B6885B0CC
:1082A000D868084B002A01D1074B1A0002920193AB
:1082B00000912B002200054900F020F800F0FAFDA3
:1082C00030020020B8A600000E9C0000C5A60000E9
:1082D000084B10B50400002B02D0002100E000BFC5
:1082E000054B1868836A002B00D09847200001F0E6
:1082F00005FBC04600000000F4A600000EB403B564
:10830000010003AB044804CB0068019300F020F99E
:1083100002B008BC03B018473002002070B5002638
:108320000C4D0D4C641BA410A64209D1002601F08F
:10833000E7FA0A4D0A4C641BA410A64205D170BD91
:10834000B300EB5898470136EEE7B300EB58984777
:108350000136F2E7000400200004002000040020A1
:108360001004002010B5034B0100186800F06AF8F3
:1083700010BDC0463002002010B5034B0100186844
:1083800000F016F810BDC04630020020002310B5E2
:108390009A4200D110BDCC5CC4540133F8E703000D
:1083A0001218934200D1704719700133F9E70000A9
:1083B00070B50500002910D00C1F2368002B00DACF
:1083C000E418280000F0A8FF1D4A1368002B05D10F
:1083D00063601460280000F0A0FF70BDA34209D9BB
:1083E000216860188342F3D118685B6841182160E6
:1083F000EEE713005A68002A01D0A242F9D91968A1
:108400005818A0420BD120680918581819608242E8
:10841000E0D110685268411819605A60DAE7A0424A
:1084200002D90C232B60D5E721686018824203D162
:10843000106852684118216062605C60CAE7C046FB
:1084400048130020032370B5CD1C9D43083506005A
:108450000C2D1ED20C25A9421DD8300000F05CFF67
:10846000254A14682100002919D1244C2368002BC7
:1084700003D1300000F02AFB20602900300000F01A
:1084800025FB431C2BD10C233000336000F045FF4B
:1084900003E0002DDFDA0C233360002070BD0B6891
:1084A0005B1B19D40B2B03D90B60CC18256003E0A0
:1084B0004B688C420DD11360300000F02EFF20007D
:1084C00007220B30231D9043C31AE7D05A42E250D3
:1084D000E4E763600C00EFE70C004968C3E703239F
:1084E000C41C9C43A042E1D0211A300000F0EEFAF7
:1084F000431CDBD1C7E7C046481300204C130020C3
:10850000936810B5013B9360002B04DA9469A34291
:1085100007DB0A2905D01368581C10601970080081
:1085200010BD00F0FBFB0100F9E7F8B506000F00F5
:108530001400D518AC4201D1002007E021783A00A0
:108540003000FFF7DDFF0134431CF3D1F8BD00001C
:10855000F0B59FB002900F0016000593002805D0DB
:1085600083690493002B01D100F0A4FD7B4B9F4253
:108570005BD1029B5F68BB891B0762D53B69002BFF
:108580005FD0002306AC6361203363761033A3769B
:1085900035002B78002B01D0252B5CD1AB1B04932D
:1085A0000CD0320039000298FFF7BFFF431C00D106
:1085B000C4E06269049B9446634463612B78002B9A
:1085C00000D1BBE0012200235242626002A9543272
:1085D00052186E1C2360E360A3601370A3653178AA
:1085E00005225F4800F07AFE751C002835D122680C
:1085F000D30604D5532302A95B1820211970130751
:1086000004D5532302A95B182B21197033782A2B28
:108610002CD0350000210A20E3682A786E1C303AFD
:10862000092A64D900292ED026E04E4B9F4202D160
:10863000029B9F689FE74C4B9F429CD1029BDF6847
:1086400099E73900029800F0BFFB002899D001207B
:1086500040421FB0F0BD01359BE7414B2268C01A74
:1086600001238340134323602E00B8E7059B191DA7
:108670001B680591002B01DB099304E05B42E3607A
:108680000223134323602B782E2B0AD16B782A2BDD
:1086900035D1059B02351A1D1B680592002B2BDB7B
:1086A0000793324E29780322300000F017FE00288D
:1086B00006D04023801B834022680135134323608A
:1086C000297806222A486E1C217600F007FE002831
:1086D0003AD0284B002B25D10722059B0733934323
:1086E000083305936369039A9B18636150E743431A
:1086F00001219B18350090E701235B42D0E700235E
:108700000A201A000135636029786E1C3039092966
:1087100003D9002BC5D00792C3E742430123521867
:108720003500F1E705AB00933A00134B21000298A6
:1087300000E000BF0390039B0133D3D1BB895B06EC
:1087400000D584E70B9884E705AB00933A000A4B09
:108750002100029800F080F8ECE7C0464CA700002A
:10876000F8A600006CA700002CA70000FEA60000E1
:1087700002A70000000000002B850000F7B51500DF
:1087800001938A680B6900900C00934200DA130091
:1087900022002B6043321278002A01D001332B6073
:1087A00023689B0602D52B6802332B6006272368BB
:1087B0001F4027D0230043331B785A1E9341226861
:1087C000920630D42200019943320098089EB047A7
:1087D000431C25D0062320682A68E1680340002551
:1087E000042B03D18D1AEB43DB171D40A3682269CC
:1087F000934201DD9B1AED180027BD4220D10020D5
:1088000010E00137E3682A689B1ABB42D2DD2200E0
:108810000123193201990098089EB047431CF0D1FA
:1088200001204042FEBD3020E11843310870210094
:108830005A1C45310978A218433202331170C1E73E
:10884000220001231A3201990098089EB047431C68
:10885000E6D00137D1E70000F0B589B004920A00F4
:1088600043320593039002920A7E0C000E9B6E2AFF
:1088700000D186E01FD8632A33D008D8002A00D15F
:108880008CE0582A4DD0250042352A7030E0642A09
:1088900001D0692AF7D1196825680A1D280629D54B
:1088A00008681A60002803DA2D23029A40421370E8
:1088B0006B4E0A274FE0732A74D008D86F2A1FD056
:1088C000702AE0D1202209680A43226003E0752A59
:1088D00016D0782AD7D12200782145321170614E06
:1088E00022E025001A684235111D196013682B70AB
:1088F000012365E008681A606906D3D500B2D1E7A4
:1089000019682568081D186008682E0605D5544E9C
:1089100008276F2A1BD00A2719E06D06F7D580B209
:10892000F5E745314E4E0A7018682268011D00684F
:108930001960150621D5D30702D520231A432260DA
:108940001027002803D1202322689A4322602300A5
:10895000002243331A706368A360002B58DB0422A3
:10896000216891432160002854D1029D002B5AD0E8
:108970002500337842352B7055E05506DBD580B2A3
:10898000D9E71A680D68101D4969186013682E062A
:1089900001D5196002E06D06FBD519800023029D08
:1089A00023614FE01A68111D196015680021626883
:1089B000280000F093FC002801D0401B6060636831
:1089C00023610023029A13703CE023692A00049972
:1089D0000398059DA847431C3ED023689B0715D4E8
:1089E000079BE068984239DA180037E0220001233B
:1089F000193204990398059EB047431C2CD00135C9
:108A0000E368079A9B1AAB42F0DCE9E70025F7E739
:108A10000028ADD0029D3900FDF79CFE735C013D3E
:108A20002B700028F7D1082F09D12368DB0706D562
:108A300063682269934202DC3023013D2B70029B64
:108A40005B1B2361059B07AA00932100049B0398ED
:108A5000FFF794FE431CB8D10120404209B0F0BD9D
:108A600009A700001AA70000124B10B51C68A36BE1
:108A7000002B0FD11820FFF775FC0F4BA06303608C
:108A80000E4B012243600E4B83600B238381002336
:108A900002614361A46B0B4A206961690A4BFDF7CF
:108AA00095FF01220023801859412061616148002F
:108AB000400810BD300200200E33CDAB34126DE6FD
:108AC000ECDE05002D7F954C2DF45158002370B538
:108AD000064C05000800236000F0FAFE431C03D199
:108AE0002368002B00D02B6070BDC0466427002097
:108AF0000CB430B5164B9DB00C1E1D6808DA8B23E4
:108B000001202B6040421DB030BC08BC02B01847A9
:108B1000822302A99B008B810023029008619C4262
:108B200000D0631E8B604B6101235B42CB81209A96
:108B300021AB2800019300F079FC431C01DA8B2360
:108B40002B60002CDFD00023029A1370DBE7C046B5
:108B5000300200200EB400B50B499CB01DAB029052
:108B60000690079104910948094904CB05910068D2
:108B700002A9019300F05AFC0023029A13701CB062
:108B800008BC03B01847C046FFFFFF7F300200203B
:108B90000802FFFF02780B78002A03D00130013170
:108BA0009A42F7D0D01A704703000A7801311A7040
:108BB0000133002AF9D170470023C25C0133002A37
:108BC000FBD1581E704730B50500002A00D130BDDA
:108BD0000C78013A6B1C2C700131002C05D19A18CD
:108BE0009A42F4D01C700133FAE71D00EDE7000053
:108BF000F0B51F000E0087B00590019102920C980D
:108C0000347800F0EAFA082200194378751C134002
:108C100036D12D2C36D1B51C74780126002F62D0A8
:108C2000102F09D1302C07D120222B789343582BB9
:108C300054D110276C7802352D4B3900F3181800E9
:108C40000393FDF787FD04910121002349420200AF
:108C50008C4618002100303909291AD80C00A74287
:108C600023DD591C09D06346824206D302D1049900
:108C7000A14202DB0123784320182C780135E9E773
:108C80002E00BCE72B2C01D01E00C7E7B51C747862
:108C9000FAE721004139192901D8373CDFE72100E3
:108CA0006139192901D8573CD9E75A1C08D1059ACE
:108CB00023331360029B0398002B09D107B0F0BD4A
:108CC000002E00D04042029A002AF7D0002B01D09B
:108CD0006B1E0193029B019A1A60EFE73024002F6C
:108CE000AAD10827A8E7302C9ED00A27A4E7C046BF
:108CF000FFFFFF7F37B51300064A05001068046ABE
:108D0000002C00D1044C0A0000942900FFF770FFEA
:108D10003EBDC0463002002094020020F8B5050098
:108D20000E001400002804D08369002B01D100F04C
:108D3000C1F9224B9C422DD16C68A369A360A38921
:108D40001B0731D52369002B2ED023682269F7B287
:108D5000981A6369F6B2834205DC2100280000F00E
:108D60003BF9002826D1A3680130013BA3602368AA
:108D70005A1C22601F706369834204D0A389DB07F9
:108D80001AD50A2E18D12100280000F025F9002854
:108D900012D00FE00A4B9C4201D1AC68CDE7094BE1
:108DA0009C42CAD1EC68C8E72100280000F00CF80A
:108DB0000028CAD0012676423000F8BD4CA700003A
:108DC0006CA700002CA70000364B70B51D6806008C
:108DD0000C00002D05D0AB69002B02D1280000F05B
:108DE00069F9314B9C420FD16C680C23E25E93B25F
:108DF00019072DD4D90611D4092301203360373344
:108E00001343A381404270BD284B9C4201D1AC6802
:108E1000EBE7274B9C42E8D1EC68E6E75B0713D50C
:108E2000616B002908D023004433994202D03000FE
:108E3000FFF7BEFA002363632422A3899343A3812F
:108E400000236360236923600823A2891343A3815D
:108E50002369002B0BD1A0218022A38989009200D5
:108E60000B40934203D02100300000F0E1F90123D0
:108E7000A289134011D00023A36063695B42A36100
:108E8000002023698342BED10C23E25E1306BAD5CB
:108E900040231343A3810138B5E7920700D46369E7
:108EA000A360EDE7300200204CA700006CA7000093
:108EB0002CA7000010B5062000F0E0FB012000F018
:108EC0001DFD0000F7B58A8905000C00130760D46A
:108ED0004B68002B04DC0B6C002B01DC0020FEBD7A
:108EE000E76A002FFAD000232E682B6080235B01F5
:108EF000216A1A4034D0606DA3895B0706D5636888
:108F0000C01A636B002B01D0236CC01A0200216AC7
:108F100000232800E76AB847A189431C06D12B68C3
:108F20001D2B30D82B4ADA40D3072CD500236360A1
:108F300023692360CB0405D5431C02D12B68002B89
:108F400000D16065616B2E600029C7D023004433D7
:108F5000994202D02800FFF72BFA00206063BEE799
:108F600001232800B847431CC6D12B68002BC3D06F
:108F70001D2B01D0162B01D12E60AFE74023A28913
:108F80001343A381ABE740230B430120A38140425D
:108F9000A5E70F69002FA1D00B680F60DB1B0193C1
:108FA0000023920700D14B69A360019B002B00DCDA
:108FB00094E7019B3A00216A2800A66AB04700287E
:108FC00003DC4023A2891343DFE7019B3F181B1AF0
:108FD0000193EAE7010040200B6970B505000C0021
:108FE000002B01D1002070BD002804D08369002B24
:108FF00001D100F05FF80B4B9C4209D16C680C2248
:10900000A35E002BEED021002800FFF75BFFEAE70C
:10901000054B9C4201D1AC68F1E7044B9C42EED178
:10902000EC68ECE74CA700006CA700002CA7000040
:10903000002310B5040003604360836081814366B0
:10904000C281036143618361190008225C30FFF72C
:10905000A6F9054B24626362044BA362044BE362EE
:10906000044B236310BDC046BD960000E59600008A
:109070001D9700004997000010B5024900F08CF8D8
:1090800010BDC046D98F000070B568254A1E5543F3
:109090000E0029007431FFF7D5F9041E08D0002115
:1090A0002A00016046600C30A0606832FFF777F953
:1090B000200070BD836913B50400002B28D18364A0
:1090C000C3640365134B144A1B6882620193984280
:1090D00001D101238361200000F020F860602000AE
:1090E00000F01CF8A060200000F018F80022E060FA
:1090F00004216068FFF79CFF01220921A068FFF7A7
:1091000097FF02221221E068FFF792FF0123A3617B
:1091100013BDC046F4A6000079900000F8B51C4BC2
:1091200007001E68B369002B02D13000FFF7C2FFB1
:109130004836B4687368013B04D53368002B07D008
:109140003668F6E70C22A55E002D0DD06834F2E7F4
:1091500004213800FFF798FF30600028F0D10C237D
:1091600004003B602000F8BD20000A4B65662560C6
:109170006560A560E36025616561A561082229003D
:109180005C30FFF70CF96563A563A564E564E9E766
:10919000F4A600000100FFFFF7B504000700002659
:1091A00001914834002C01D13000FEBD6368A568F0
:1091B0000093009B013B009301D52468F2E7AB8943
:1091C000012B08D90E22AB5E013304D029003800F0
:1091D000019B984706436835EBE7EC300068704721
:1091E00070B50E001D000E23C95E96B01400002954
:1091F00007DA00232B60B3891B0611D48023DB0020
:109200000FE06A4600F0D8FA0028F2DBF022019B5A
:1092100012021340054A9B185A4253412B60EDE756
:1092200040230020236016B070BDC04600E0FFFF61
:10923000F7B502268B8905000C00334206D02300C7
:1092400047332360236101236361F7BD01AB6A46A5
:10925000FFF7C6FF009907002800FFF7F3F8002882
:1092600008D10C22A35E9A05EFD4032293431E4338
:10927000A681E4E70F4BAB628023A28920601343F1
:10928000A381009B20616361019B002B0DD00E2305
:10929000E15E280000F0A2FA002806D00322A3898C
:1092A00093431A0001231343A381A0893843A0816B
:1092B000CBE7C0467990000082B0002900D101A917
:1092C000101E06D0002B06D013780B601078431EBA
:1092D000984102B0704702204042FAE7C9B28218B2
:1092E000904201D10020704703788B42FBD00130BF
:1092F000F6E710B5884202D98B18984203D30023B1
:1093000007E08B5C8354013AFBD210BDCC5CC454A3
:1093100001339A42FAD1F8E770477047F8B5070071
:109320000D001600002905D11100FFF78BF804008D
:109330002000F8BD002A03D1FFF73AF83400F7E720
:1093400000F072FA2C00B042F2D231003800FFF780
:1093500079F8041EECD029003200FFF717F8290035
:109360003800FFF725F8E3E7F0B58E6885B0070011
:109370000C00039201939E423CD890238A89DB0023
:109380001A4234D00325096923685B1A0293636982
:1093900002985D43EB0F5D19019B6D1001331B18A3
:1093A000AB4200D91D00530532D529003800FFF724
:1093B00049F8061E09D10C233B6040230120A289F5
:1093C00040421343A38105B0F0BD029A2169FEF724
:1093D000DDFFA389144A1A4080231343A381029B13
:1093E0002661F61826606561019EED1AA560019B55
:1093F0009E4200D9019E320003992068FFF779FF51
:10940000A36800209B1BA36023689E192660DAE7EF
:109410002A003800FFF782FF061EE0D121693800DC
:10942000FEF7C6FFC7E7C0467FFBFFFFF0B59FB062
:10943000029005938B890F0016001B0611D50B694E
:10944000002B0ED14021FEF7FDFF38603861002867
:1094500005D10C23029A013813601FB0F0BD4023E0
:109460007B61002306AC6361203363761033A376FF
:1094700035002B78002B01D0252B46D1AB1B049354
:109480000CD0320039000298FFF76EFF431C00D168
:10949000AEE06269049B9446634463612B78002BC1
:1094A00000D1A5E0012200235242626002A9543299
:1094B00052186E1C2360E360A3601370A3653178BB
:1094C00005225448FFF70AFF751C00281FD12268A7
:1094D000D30604D5532302A95B1820211970130762
:1094E00004D5532302A95B182B21197033782A2B3A
:1094F00016D0350000210A20E3682A786E1C303A25
:10950000092A4ED9002918D010E00135B1E7414BA6
:109510002268C01A01238340134323602E00CEE744
:10952000059B191D1B680591002B01DB099304E0C5
:109530005B42E3600223134323602B782E2B0AD176
:109540006B782A2B35D1059B02351A1D1B680592B5
:10955000002B2BDB0793304E297803223000FFF7D6
:10956000BDFE002806D04023801B834022680135C1
:10957000134323602978062228486E1C2176FFF7C2
:10958000ADFE00283CD0264B002B25D10722059BA1
:1095900007339343083305936369039A9B18636108
:1095A00066E7434301219B183500A6E701235B4290
:1095B000D0E700230A201A000135636029786E1C69
:1095C0003039092903D9002BC5D00792C3E742439C
:1095D000012352183500F1E705AB00933A00114B17
:1095E0002100029800E000BF0390039B0133D3D118
:1095F000BB890B985B0600D42FE7012040422CE783
:1096000005AB00933A00074B21000298FFF724F9BD
:10961000EAE7C046F8A60000FEA6000002A7000088
:10962000000000006993000070B504000D001F29C0
:1096300004D9162303600120404270BD436C002B07
:1096400004D08A009B181A68002A08D1200000F074
:1096500031F82A000100200000F01AF8EDE70020A0
:10966000012AEAD0511C03D1162301302360E4E71C
:10967000002428001C6090472000DEE710B5034B53
:1096800001001868FFF7D0FF10BDC046300200206F
:10969000002370B5064C050008001100236000F09F
:1096A000FFF8431C03D12368002B00D02B6070BD52
:1096B0006427002010B500F0E3F810BD70B50C0071
:1096C0000E25495F00F0B8F8002803DB636D1B1816
:1096D000636570BDA389024A1340A381F9E7C046C0
:1096E000FFEFFFFFF8B51F008B8905000C00160087
:1096F000DB0505D50E23C95E0022022300F080F8A9
:10970000A389054A28001340A38132000E23E15E9D
:109710003B0000F02BF8F8BDFFEFFFFF70B50C0029
:109720000E25495F00F06CF8A389421C03D1054A5D
:109730001340A38170BD802252011343A381606551
:10974000F8E7C046FFEFFFFF10B50E23C95E00F03B
:1097500021F810BD0B1E04D0FF2A04D98A23036010
:109760008B3B180070470A700123FAE770B50500BB
:10977000080011000022064C22601A0000F0B6F822
:10978000431C03D12368002B00D02B6070BDC04662
:1097900064270020002370B5064C050008002360F4
:1097A00000F05EF8431C03D12368002B00D02B602F
:1097B00070BDC04664270020002370B5064C05002C
:1097C00008001100236000F053F8431C03D1236804
:1097D000002B00D02B6070BD64270020002370B5E3
:1097E000064C05000800236000F052F8431C03D12A
:1097F0002368002B00D02B6070BDC046642700207A
:1098000070B50500080011000022064C22601A0005
:1098100000F04EF8431C03D12368002B00D02B60CE
:1098200070BDC046642700200B1F1B68181F002B4B
:1098300001DA0B58C018704770B505000800110018
:109840000022064C22601A0000F03AF8431C03D1B3
:109850002368002B00D02B6070BDC0466427002019
:1098600058220120014B40421A60704764270020B3
:1098700058220120014B40421A60704764270020A3
:1098800058220120014B40421A6070476427002093
:109890005822024B00201A607047C04664270020FF
:1098A00058220120014B40421A6070476427002073
:1098B00058220120014B40421A6070476427002063
:1098C00058220120014B40421A6070476427002053
:1098D000044A1368002B00D1034B181810601800BD
:1098E0007047C046501300206827002058220120EE
:1098F000014B40421A60704764270020FEE7C046D3
:10990000F8B5C046F8BC08BC9E467047F8B5C046DE
:10991000F8BC08BC9E46704750050000600500007A
:109920007A050000F8050000300600006606000019
:109930009E060000C4060000000700004207000069
:1099400098070000DC0700004808000090080000AD
:10995000B6080000EE080000340900005A090000B3
:1099600088090000BA090000F2090000760A000028
:10997000420B0000B80B0000240C00006C0C00002F
:109980008C0C0000AE0C0000880D0000CE0D000015
:10999000500500005005000050050000460E000074
:1099A000AE0E0000300F0000760F0000BE0F00006A
:1099B0003C100000BA100000021100004811000025
:1099C0007E110000C41100000A12000052120000B3
:1099D000A61200000413000042130000AC130000A4
:1099E000E21300002A14000072140000BA140000F0
:1099F000F41400003C150000841500005005000020
:109A00005005000050050000EC1500002216000073
:109A10005816000084160000BA160000F016000068
:109A200050050000500500005005000050050000E2
:109A300026170000681700005005000050050000C0
:109A4000AE170000FE1700002418000050050000AB
:109A50005005000050050000521800008218000058
:109A6000B2180000E21800000C19000042190000B2
:109A70006C19000094190000BC190000EC190000DA
:109A80001C1A0000461A0000701A0000A01A0000FC
:109A9000E41A0000500500005005000050050000C9
:109AA0005005000050050000141B0000401B000082
:109AB0006C1B0000981B0000C41B0000FA1B000078
:109AC000301C0000661C00009C1C0000C81C00002C
:109AD000F41C00002A1D0000500500005005000085
:109AE0005005000050050000500500005005000022
:109AF0005005000050050000500500005005000012
:109B00005005000050050000500500005005000001
:109B1000561D0000821D000066616C736500747242
:109B20007565006C697374206F6620256420697404
:109B3000656D73006F626A656374206F6620636C85
:109B40006173733A20256400537461636B20756EF2
:109B5000646572666C6F7700070000000300000008
:109B600015000000010000000200000004000000D9
:109B7000050000000600000043616C6C696F7065B1
:109B800000686173546F6E6500706C6179546F6E1C
:109B90006500686173536572766F00736574536511
:109BA00072766F00496E73756666696369656E7477
:109BB000206D656D6F727920666F72204D696372DA
:109BC0006F426C6F636B73206F626A6563742068A9
:109BD00065617000496E73756666696369656E7468
:109BE000206D656D6F727920666F72204D696372AA
:109BF0006F426C6F636B7320737461636B000D0A4B
:109C0000564D2050616E69633A2025730D0A006D30
:109C100069736300686578546F496E740073696E88
:109C2000006E6574006861735769466900737461FA
:109C30007274576946690073746F7057694669009A
:109C400077696669537461747573006D7949504121
:109C5000646472657373007468696E6744657363E6
:109C600072697074696F6E00636C656172546869C3
:109C70006E674465736372697074696F6E006170BA
:109C800070656E64546F5468696E6744657363727F
:109C9000697074696F6E00617070656E64546F54A2
:109CA00068696E6750726F7065727479000D0E0F7F
:109CB00004050C0B0A0607080904050C0B0A060725
:109CC0000809000000000008080800080A4A4000CF
:109CD000000A5FEA5FEA0ED92ED36E193244893347
:109CE0000C924C924D0808000000048808080408F3
:109CF00004848488000A448A4000048EC4800000E2
:109D000000048800000EC00000000008000122448A
:109D100088100C9252524C048C84848E1C824C907D
:109D20001E1EC244924C06CA525FE21FF01EC13E84
:109D300002448ED12E1FE24488100ED12ED12E0E59
:109D4000D12EC48800080008000004800488024462
:109D5000880482000EC00EC008048244880ED126FA
:109D6000C0040ED135B36C0C925ED2521C925C9240
:109D70005C0ED010100E1C9252525C1ED01C901E15
:109D80001ED01C90100ED013712E12525ED2521C97
:109D90008808081C1FE242524C125498149210106A
:109DA00010101E113B75B131113935B3710C92523F
:109DB000524C1C925C90100C92524C861C925C92FD
:109DC000510ED00C825C1FE4848484125252524C97
:109DD0001131312A44113135BB7112524C9252115A
:109DE0002A4484841EC488101E0EC808080E100859
:109DF0000482410EC242424E048A4000000000002C
:109E0000001F0804800000000ED2524F10101C9258
:109E10005C000ED0100E02424ED24E0C925C900EA0
:109E200006C81C88080ED24EC24C10101C92520854
:109E300000080808024002424C10149814920808C6
:109E4000080806001B75B131001C925252000C929A
:109E5000524C001C925C90000ED24EC2000ED010EC
:109E6000100006C8049808080EC807001252524F86
:109E70000011312A4400113135BB00124C8C920084
:109E8000112A4498001EC4881E06C48C84860808C3
:109E900008080818080C881800000C8360000000EF
:109EA00000000000010000000200000003000000AC
:109EB000040000000500000006000000070000008C
:109EC00008000000090000000A0000000B0000006C
:109ED0000C0000000D0000000E0000000F0000004C
:109EE0001000000012000000140000001600000026
:109EF000180000001A0000001C0000001E000000F6
:109F000020000000230000002600000029000000BF
:109F10002C0000002F00000032000000360000007E
:109F20003A0000003E000000420000004600000031
:109F30004B00000050000000550000005A000000D7
:109F400061000000680000006F0000007600000063
:109F50007D000000840000008B00000092000000E3
:109F600099000000A0000000A7000000AE00000063
:109F7000B5000000BC000000C3000000CA000000E3
:109F8000D1000000D8000000DF000000E600000063
:109F9000ED000000F4000000FB000000FF000000E6
:109FA000646973706C6179006C696768744C65767C
:109FB000656C006D62446973706C6179006D624418
:109FC0006973706C61794F6666006D62506C6F7476
:109FD000006D62556E706C6F74006D6244726177D3
:109FE0005368617065006D625368617065466F7299
:109FF0004C6574746572006E656F506978656C535A
:10A00000656E64006E656F506978656C5365745059
:10A01000696E004E6F7420656E6F75676820726F91
:10A020006F6D206576656E20616674657220636F62
:10A030006D70616374696F6E0A00436F6D70616368
:10A0400074656420466C61736820636F6465207377
:10A05000746F72650A256420627974657320757364
:10A06000656420282564252529206F662025640045
:10A07000426164207265636F726420666F756E64FE
:10A0800020647572696E6720696E697469616C69B4
:10A090007A6174696F6E210A002564202564202589
:10A0A000642028256420776F72647329002564205A
:10A0B0007265636F7264732C20256420776F7264FD
:10A0C000732C206D617849442025642C20636F6DCA
:10A0D00070616374696F6E206379636C65732025AA
:10A0E00064005363726970747320636C6561726598
:10A0F00064005374617274656400526573746F72A6
:10A1000065642025642073637269707473007261E2
:10A1100064696F006E6F6E650064697361626C657F
:10A12000526164696F006D65737361676552656341
:10A130006569766564007061636B6574526563651B
:10A14000697665007061636B657453656E64007257
:10A1500065636569766564496E74656765720072EA
:10A16000656365697665644D657373616765547988
:10A170007065007265636569766564537472696EB3
:10A18000670073656E64496E746567657200736518
:10A190006E64506169720073656E64537472696EA7
:10A1A00067007365744368616E6E656C00736574F7
:10A1B00047726F757000736574506F7765720073C6
:10A1C00069676E616C537472656E67746800416C88
:10A1D0006C207461736B732073746F7070656400AE
:10A1E0007630363500202573202573004D656D6F60
:10A1F000727920636C6561726564004E6F206672CF
:10A200006565207461736B20656E74726965730097
:10A2100073656E736F72730074656D7065726174CF
:10A220007572650074696C74580074696C745900B7
:10A2300074696C745A00746F756368526561640068
:10A24000693263526561640069326357726974658B
:10A250000074667400656E61626C65446973706C4D
:10A26000617900676574576964746800676574484C
:10A27000656967687400736574506978656C006C13
:10A28000696E65007265637400726F756E646564F3
:10A290005265637400636972636C6500747269610E
:10A2A0006E676C65007465787400746674546F75BD
:10A2B0006368656400746674546F756368580074ED
:10A2C0006674546F7563685900746674546F75636F
:10A2D0006850726573737572650057656C636F6D56
:10A2E0006520746F204D6963726F426C6F636B738E
:10A2F0002100705F73706920213D204E554C4C0049
:10A300002F686F6D652F62726F6D61676F73612F5C
:10A310002E706C6174666F726D696F2F7061636B04
:10A32000616765732F6672616D65776F726B2D6102
:10A33000726475696E6F6E6F726469636E72663592
:10A340002F6C69627261726965732F5350492F5384
:10A3500050492E63707000535049436C6173733AD7
:10A360003A535049436C617373284E52465F5350C1
:10A37000495F547970652A2C2075696E74385F7452
:10A380002C2075696E74385F742C2075696E743872
:10A390005F74290000000000000000007546000006
:10A3A0003146000057460000614600006B46000041
:10A3B00055460000000000000100000002000000FF
:10A3C0001600000004000000050000000600000068
:10A3D0000700000008000000090000000A0000005B
:10A3E0000B0000000C0000000D0000000E0000003B
:10A3F0000F0000001A0000001B0000001400000005
:10A400001300000011000000030000001000000015
:10A410001C0000001D0000001E00000012000000D3
:10A4200015000000170000001800000019000000CF
:10A4300000000000000000007D4B000061490000AA
:10A44000FD4B0000114C0000074C0000794B000050
:10A450006D4B00001D4C0000994B0000694B000043
:10A46000FB21F93FFB2109407CD91240FB21194017
:10A470007A6A1F407CD92240BBFD2540FB21294040
:10A480003A462C407A6A2F405C4731407CD93240B2
:10A490009C6B3440BBFD3540DB8F3740FB2139409E
:10A4A0001BB43A403A463C405AD83D407A6A3F4055
:10A4B0004C7E40405C4741406C1042407CD9424059
:10A4C0008CA243409C6B4440AC344540BBFD4540AE
:10A4D000CBC64640DB8F4740EB584840FB21494004
:10A4E00083F9A200444E6E00FC291500D1572700C5
:10A4F000DD34F50062DBC0003C99950041904300DB
:10A500006351FE00BBDEAB00B761C5003A6E2400AC
:10A51000D24D42004906E00009EA2E001C92D1000B
:10A52000EB1DFE0029B11C00E83EA700F5358200B6
:10A5300044BB2E009CE98400B4267000417E5F007D
:10A54000D6913900538339009CF439008B5F840025
:10A5500028F9BD00F81F3B00DEFF97000F980500AB
:10A56000112FEF000A5A8B006D1F6D00CF7E360051
:10A5700009CB2700464FB7009E663F002DEA5F00DB
:10A58000BA277500E5EBC7003D7BF100F7390700FE
:10A5900092528A00FB6BEA001FB15F00085D8D00DC
:10A5A000300356007BFC4600F0AB6B0020BCCF00B4
:10A5B00036F49A00E3A91D005E619100081BE600D5
:10A5C00085996500A0145F008D40680080D8FF0069
:10A5D00027734D0006063100CA561500C9A873003E
:10A5E0007BE260006B8CC00000000040FB21F93F63
:10A5F000000000002D44743E000000809846F83CA6
:10A600000000006051CC783B00000080831BF039D3
:10A610000000004020257A38000000802282E336C6
:10A62000000000001DF36935020000000300000077
:10A630000400000006000000186B0000C26A000061
:10A64000C26A0000F06B0000BE6A0000BE6A000033
:10A65000E66B0000F06B0000BE6A0000E66B0000D5
:10A66000BE6A0000F06B0000F46B0000F46B0000A9
:10A67000F46B0000FC6B0000187700001A760000F5
:10A680001A76000038790000147600001476000075
:10A69000207900003879000014760000207900004D
:10A6A00014760000387900002E7900002E79000021
:10A6B0002E7900003C7900002C2066756E63746969
:10A6C0006F6E3A2000617373657274696F6E202239
:10A6D000257322206661696C65643A2066696C6541
:10A6E00020222573222C206C696E65202564257339
:10A6F00025730A0034020020232D302B2000686CC3
:10A700004C00656667454647003031323334353694
:10A7100037383941424344454600303132333435CD
:10A7200036373839616263646566000000000000F6
:10A730000000000000000000000000000000000019
:10A740000000000000000000000000000000000009
:10A7500000000000000000000000000000000000F9
:10A7600000000000000000000000000000000000E9
:10A7700000000000000000000000000000000000D9
:10A780000000000000000000000000004300504FE7
:10A79000534958002E000020202020202020202077
:10A7A0002828282828202020202020202020202081
:10A7B00020202020202020881010101010101010B1
:10A7C00010101010101010040404040404040404F5
:10A7D000041010101010101041414141414101017D
:10A7E0000101010101010101010101010101010159
:10A7F0000101101010101010424242424242020267
:10A800000202020202020202020202020202020228
:10A8100002021010101020000000000000000000D4
:10A820000000000000000000000000000000000028
:10A830000000000000000000000000000000000018
:10A840000000000000000000000000000000000008
:10A8500000000000000000000000000000000000F8
:10A8600000000000000000000000000000000000E8
:10A8700000000000000000000000000000000000D8
:10A8800000000000000000000000000000000000C8
:0CA89000000000000000000000000000BC
:08A89C006C58FF7F0100000071
:10A8A400FFFFFFFF40060000819B00005D1E0000CB
:10A8B400899B0000611E0000929B0000591E00004D
:10A8C4009B9B0000651E0000149C0000A122000058
:10A8D4001D9C0000F5220000259C0000D1230000EF
:10A8E4002D9C0000D5230000379C0000F3230000BA
:10A8F400409C0000FD2300004B9C00000724000046
:10A90400579C000011240000689C00001B240000D8
:10A914007E9C0000DF230000979C0000E9230000D8
:10A92400A89F000041240000B39F00000D290000EF
:10A93400BD9F000021260000CA9F000041260000A0
:10A94400D19F000091260000DA9F0000E12600005C
:10A95400E69F000039290000F79F000051280000FD
:10A9640004A00000212800001800000019A1000024
:10A974002533000026A100006533000036A1000045
:10A984006933000044A100006D3300004FA10000B2
:10A99400293300005FA100003D33000073A10000D3
:10A9A4002D33000082A10000713300008EA100004D
:10A9B4007533000097A1000079330000A2A10000C4
:10A9C4007D330000ADA100005D330000B6A100009E
:10A9D40061330000BFA100003533000018A200005D
:10A9E4003943000024A20000554300002AA20000BD
:10A9F4008543000030A200000743000036A2000097
:10AA0400C540000040A20000B543000048A2000079
:10AA1400F141000055A200003944000063A2000087
:10AA2400454400006CA200004944000076A20000E6
:10AA34004D4400007FA200005144000084A20000A5
:10AA44005544000089A200005944000095A200006A
:10AA54005D4400009CA2000061440000A5A2000027
:10AA640065440000AAA2000069440000B5A20000E9
:10AA74006D440000BFA200003D440000C9A20000D4
:10AA8400414400000200000003000000FFFFFFFF3C
:10AA940000000000010000000000020001000000AE
:10AAA400FFFFFFFF000000000200000000000400A0
:10AAB40002000000FFFFFFFF000000000300000091
:10AAC40000000800030000000A0000000800000065
:10AAD40034020020000000004CA700006CA7000016
:10AAE4002CA700000000000000000000000000008F
:10AAF4000000000000000000000000000000000052
:10AB04000000000000000000000000000000000041
:10AB14000000000000000000000000000000000031
:10AB24000000000000000000000000000000000021
:10AB340000000000430000000000000000000000CE
:10AB44000000000000000000000000000000000001
:10AB540000000000430000000000000000000000AE
:10AB640000000000000000000000000000000000E1
:10AB7400000000004300000000000000000000008E
:10AB840000000000000000000000000000000000C1
:10AB9400000000004300000000000000000000006E
:10ABA40000000000000000000000000000000000A1
:10ABB400000000004300000000000000000000004E
:10ABC4000000000000000000000000000000000081
:10ABD400000000004300000000000000000000002E
:10ABE4000000000000000000000000000000000061
:10ABF400000000004300000000000000000000000E
:10AC04000000000000000000000000000000000040
:10AC14000000000055970000B992000000000000F9
:10AC240096A7000094A700000E9C00000E9C000054
:10AC34000E9C00000E9C00000E9C00000E9C000068
:10AC44000E9C00000E9C00000E9C0000FFFFFFFF06
:10AC5400FFFFFFFFFFFFFFFFFFFF00000100415365
:10AC6400434949000000000000000000000000000B
:10AC7400000000000000000000000000000041533C
:10AC840043494900000000000000000000000000EB
:10AC940000000000000000000000000000000000B0
:10ACA400E90000000146000049490000C94E0000C7
:04ACB400C1000000DB
:0400000300004A3D72
:00000001FF
